:10000000400E0020F1000000C1000000C10000000F
:1000100000000000000000000000000000000000E0
:10002000000000000000000000000000C10000000F
:100030000000000000000000C1000000C10000003E
:10004000BD5800001D060000E94D0000054E0000EF
:10005000694D00009D4D000021510000E951000054
:100060006D600000D501000015020000550200007F
:10007000490600009D770000C1000000C10000009B
:10008000C1000000C1000000C1000000C10000006C
:10009000C1000000C1000000C1000000C10000005C
:1000A000C1000000C1000000C1000000C10000004C
:1000B00029590000F9B70000C1000000C10000008C
:1000C00010B500F04FFD0321064A13680B4313607F
:1000D000054A064B02391A60A022D20593680B43E9
:1000E0009360FEE700C000500400FA050CED00E04C
:1000F000002370B50A480B490B4C1A188A4203D2E8
:10010000E55804331560F8E70021084B084A93428C
:1001100001D202C3FBE707F04FFE00F099FE70BD6D
:100120000000002034000020F0BE00003400002059
:10013000400A0020002307B5019303281DD8114B66
:1001400002301A6880000723C2401A406B4603330E
:100150001A701A78002A02D105F0F6FB04E01A782A
:10016000022A03D105F026FC019004E01B78072B3E
:1001700005D1054B0193019802E0044800E00448D2
:100180000EBDC04614020050008051010197FFFFD0
:100190000297FFFFF8B507000E00012815D90029C6
:1001A00013D001240D00290038000BF0F9FB084A98
:1001B000831E934203D8013C2406204307E080239A
:1001C0000134AD195B009C42EDD101204042F8BDE5
:1001D000FDFFFF00012110B50C4A0D4C93680B4345
:1001E000936023685B1823606368002B0CD0A368BE
:1001F000002B09D02369013B2361002B04D16369E3
:10020000A0699847E368236110BDC0462000014003
:1002100034000020012110B50C4A0D4C93680B43AB
:100220009360E3695B18E361236A002B0CD0636A77
:10023000002B09D0E36A013BE362002B04D1236B5E
:10024000606B9847A36AE36210BDC046000011408E
:1002500034000020012110B50C4A0D4C93680B436B
:100260009360A36B5B18A363E36B002B0CD0236C30
:10027000002B09D0A36C013BA364002B04D1E36CD9
:10028000206D9847636CA36410BDC04620001140E8
:10029000340000200122034B5A659A65DA651A661C
:1002A0007047C04634000020F7B50C000190009262
:1002B000032800D97FE0434B0BF05EFB02203F5642
:1002C000596D012979D1586E002876D104273E4E08
:1002D0005966B2683A43B2603C4E3060B2680A4335
:1002E000B260D86798663A4B1C60FFF723FF210085
:1002F000FFF750FF431C4ED1364861E0986D01284E
:100300005BD133494A68002A57D108252E4F4860EF
:10031000BE682E43BE60304E3260B7680743B76098
:100320009A601A608C60FFF705FF2100FFF732FF2B
:10033000431CE1D00302EB402FE0D86D01283CD1F3
:100340002349CA68002A38D110251F4FC860BE68EB
:100350002E43BE60214E3260B7683843B060DA6128
:100360005A620C610220C0E7186E012825D1184995
:100370004A69002A21D12025134F4861BE682E43C7
:10038000BE60174E3260B7683843B0609A631A6433
:100390008C610320A9E703021B0A7360009B000E17
:1003A000DB061843009B3060022B08D101980F3008
:1003B000C0B204F0C3FD0B4802E00B4800E000208F
:1003C000FEBDC04634000020000200500000014085
:1003D000B40000200297FFFF200001400000114000
:1003E000200011400197FFFF0397FFFF73B5002422
:1003F000032800D9C6E0644C0BF0BEFA02326493C5
:10040000E569002D00D0BCE0012014262062E069DF
:100410000130E0615D4C0195019800282FDC019DC1
:10042000142075436519AD6E002D15D10126019D6F
:1004300045436519AE66019D45436519E966019D11
:100440004543651929670199414361184A67019A33
:1004500050432018836792E0019801300190DBE758
:10046000666A002E00D08CE0012548484560656A28
:100470000135656201961436019C002C01DD0024D3
:1004800080E0019D142475434519AD68002D15D1F8
:100490000126019D65434519AE60019D65434519DF
:1004A000E960019D6543451929610199614341183E
:1004B0004A61019A54430019836160E0019C013450
:1004C0000194D9E7A66A002E5BD101252F48056269
:1004D000A56A0135A56201961436019C002CCEDC7C
:1004E000019D1424754345196D6A002D15D101260F
:1004F000019D654345196E62019D65434519A962D9
:10050000019D65434519E9620199614341180A63F8
:10051000019A54430019436331E0019C0134019472
:10052000DBE7E66A002E2CD101251848C563E56A91
:100530000135E5620196143602E0019C0134019414
:10054000019C002C9BDC019D1424754345192D6CE6
:10055000002DF2D10126019D654345192E64019DB0
:10056000654345196964019D65434519A96401996D
:1005700061434118CA64019A544300190365019C00
:1005800000E0034C200076BDB400002034000020C1
:100590000497FFFF30B503281FD88021104B82003D
:1005A000D358104A89059B181A6808300A431A6004
:1005B0000323FF22C0B2C2240340DB009A400A4951
:1005C000A4000D59954380229A4013002B430B51F0
:1005D0000123834000200B6000E0044830BDC0468A
:1005E0008CBC00000000014000E100E00197FFFF2B
:1005F00003280BD88021064B8000C358054AC90543
:100600009B181A6800200A431A6000E002487047ED
:100610008CBC0000000001400197FFFF07B50821D6
:10062000074A13689B06DB0F019313680B431360A3
:10063000044B1B6B002B01D00198984707BDC046A7
:1006400000400040B4000020044B10B51868044B73
:100650001B68002B00D0984710BDC0461C00054009
:10066000E8000020824BF7B50D00184200D0F3E0FF
:100670008A79072A00D9F1E0AB23D340DB0700D405
:10068000ECE00B79032B00D9EAE04B79012B00D980
:10069000E8E0CB79062B00D9E6E0A023DB0575491D
:1006A000DA688024002805D164022243DA60DE681B
:1006B000714A04E0A4022243DA60DE686F4A3240E5
:1006C000DA608B680F2623438B606D4BC4180420BF
:1006D000A3680343A3600223A2681A43A260EF79D0
:1006E000A2683E40F0278640BA433243A260AE790A
:1006F000D03F0640721E9641E2687601BA4332430B
:10070000E260AA79E76813405A1E93411A01102348
:100710009F433B00012608271343E360AA79E3685F
:100720003240D200BB431343E360E3682A79053FBC
:100730003A40BB431343E360E2686B7982431E4057
:10074000B30016001E43E660236A2A7AFB30834317
:10075000134323620A68474BD20703D55869494AB5
:1007600002400FE01A6AD20305D45869454A024094
:100770008020400405E01A68520777D5C0205A69E6
:10078000800402435A618E694B693605360F9B011E
:100790009B0F0136002B02D105F0D6F807E0354B50
:1007A0005B699B019B0F012B03D105F0D1F8310050
:1007B00001E0310034480BF0F3F82F6806003900EF
:1007C0000BF0EEF80F2305000340626A012B0CD8F2
:1007D0007F01B74209D22D4B050913406362626A5B
:1007E0002B4BAF1E134063622EE0802180238905CE
:1007F0000A436262626A5B051A43264BAF1E62625D
:100800009F4221DD0826636A0B436362626A204BC4
:1008100013406362731C1900280001930BF046F922
:1008200002290ED80F23616A1B4A1E40114033066D
:100830000E001E436662019928000BF0B1F8871E76
:1008400002E0019E102EE5D1656AB8B22D0C2D0490
:100850000543656200200AE0104808E0104806E001
:10086000104804E0104802E0104800E01048FEBDC7
:10087000FFFFEFFF00020050FFFFFEFFFFFFFDFF45
:1008800000000540FFFFFFFC00805101FFFFFFDF7C
:10089000FFFFFFEFFFFF0000FFFFFFF00298FFFFE9
:1008A0000398FFFF0498FFFF0598FFFF0698FFFFDE
:1008B0000898FFFFF7B501240E002E4B0192C318D4
:1008C0005D682640A54335434E0802272640A640D2
:1008D0005D605D68BD4335438E082640BE405D6067
:1008E0005D68FF19BD4335435D605D68CE082640F5
:1008F0000437F600BD4335435D605E680D09B446BC
:1009000062461D4E2540EF0216403E4310275E60B2
:100910005E682D01BE4335434E09890926400C40CF
:10092000A10140245D605D68FF197601BD43354338
:100930005D605D68A5432C000C43C3215C608900A9
:100940000E4B00280BD1019A0D480260FF205A5827
:1009500082437F3802435A508022520108E058589F
:10096000084A02408020000202435A50802292012D
:100970001A60F7BD00000540FFF7FFFF00E100E04F
:10098000E8000020FF00FFFF0322F0B5214B224EBC
:10099000C018036B214F134303634C780123621E7D
:1009A0009441C56A1E4AE4032A402243C262C56AD2
:1009B0008A7814062A02120A2243C2620C78C26A9A
:1009C0001C40324024022243C2620C78C26ADC40DE
:1009D000144D1C4064022A402243C2620C78C26A51
:1009E000A4081C40A4023A402243C262076ACC78A1
:1009F0000D4A24023A40224302620A798168134078
:100A00001A020B0033401343836003691D400561E4
:100A1000F0BDC04600000540FFFEFFFFFFFBFFFFEB
:100A2000FF7FFFFFFFFDFFFFFF00FFFF30B50F243B
:100A30000125124BDA68A2432A43DA60DA686419A6
:100A4000A243DA602022DC681443DC6058609960BD
:100A50001A692A431A61BFF36F8F1869074AC007E2
:100A6000C00FC0B20028F8D113685B0604D540213E
:100A7000136803480B43136030BDC04600C00050EC
:100A80008188FFFF10B50F24134BDA68A243DA60A8
:100A9000DA680134A243DA60DA681034A243DA601B
:100AA0000022586001209A601A6902431A61BFF35C
:100AB0006F8F1869084AC007C00FC0B20028F8D16C
:100AC00013685B0605D54021136804480B43136087
:100AD00001E093680B6010BD00C000508188FFFFEB
:100AE0000F21124BDA688A430D390A43DA60DA685B
:100AF0000E318A43DA60DA6810310A43DA605860EE
:100B00001A691F390A431A61BFF36F8F1869074AC0
:100B1000C007C00FC0B20028F8D113685B0604D527
:100B20004021136802480B431360704700C0005017
:100B30008188FFFF0421054A53680B435360044A30
:100B4000033913680B4313607047C046000200501E
:100B500000C000500121024A13688B4313607047A4
:100B600000C0005010B5162059248821034B5C604A
:100B7000586059605A68002AF9D010BDFC00005036
:100B800073B504000E00FFF7EDFFFFF7D3FFF82366
:100B9000DB01E518AD0001A92800FFF773FF019BF9
:100BA00033409E4204D131002800FFF73FFF14E09C
:100BB000F8204002FFF794FF0B4D640066530024B9
:100BC0006300E95A094BC918F823DB01E0188000DB
:100BD0000134FFF72BFF802CF2D1FFF7BBFF04F0AD
:100BE00057FE002076BDC046200200200000FFFF17
:100BF000F0B5441CE4B285B00D00632C11D9642615
:100C0000200031000AF052FF434BCCB26200D05AB0
:100C1000310080B20AF04AFF7543ADB269188DB257
:100C200013E02738182810D83B4B6200D05AD35A0B
:100C300080B299B22B1C632D00D96323CB18642199
:100C40009DB20AF033FF6D1AADB223001F3B012B9A
:100C50005FD9082C09D1FFF785FFFFF76BFFF8205C
:100C60004002FFF73DFF2D4854E02B4E6300985B98
:100C7000019380B285424DD0FFF774FF8022284B4C
:100C80009201DA67FFF756FFF823DB01E418A400AE
:100C900003A92000FFF7F6FE039B10272B409D427F
:100CA00009D1204B2000E9180391FFF7BFFE1EE099
:100CB000013F002F1BD0F8204002FFF711FFF82062
:100CC00003A94002FFF7DEFE039B0133F0D10027AA
:100CD000019BF5527B00F15A124BC918F823DB0136
:100CE000F81880000137FFF7A1FE802FF2D103A989
:100CF0002000FFF7C7FE039B9CB2FFF72BFF80226B
:100D0000094B92011A6004F0C3FD019B2000F552CB
:100D100000E0064805B0F0BD20020020FEFF000004
:100D200004E100E00000FFFF00E100E0FFFF000041
:100D3000044B4118884203D0027801301A60F9E769
:100D40007047C046000005408021104B09011A6819
:100D5000F0B50A431A6000211A000D4D0D4E0E4FDA
:100D60006B5C28009C46735C34009C4502D0136881
:100D70003B40136001311029F2D10023E25CD2B272
:100D8000C2540133102BF9D1F0BDC04668070020D2
:100D9000A204002061040020FFF7FFFF0821074B99
:100DA0009A680A439A60064A02391180118800291C
:100DB000FCD19A6808318A439A607047004000501D
:100DC0009A04002010B540240F4A9368A34393600F
:100DD000072817D803234B430AF0CEFD0406080A60
:100DE0000C0E1012094A0CE0094A0AE0094A08E010
:100DF000094A06E0094A04E0094A02E0094A00E01B
:100E0000094A136010BDC046C040005010000440A5
:100E10001C000440100014401C0014402800044032
:100E200034000440280014403400144010B58842B7
:100E300001D9401A00E0081A0A23534380B219006E
:100E40000AF038FEFF23984200DCC3B2180010BD40
:100E5000F0B5D54BD54FD64E3B60D64BD64D336013
:100E6000D64BD74C2B60D74BD74A2360D74B97B084
:100E70001A600023D54A93605822BB60B360AA6011
:100E8000D34AA36011681360FFF76CFE0121D14BB8
:100E90001A680A431A6009961E00C34A08970B9203
:100EA000CA4A04950792C84A0C940A92F368C94A40
:100EB000DB07FBD5116AC84B01200B4013620C23E2
:100EC000C64A1360BC3311681943014204D111684A
:100ED0005B0849081160F6E7C02112680902023A6E
:100EE0005202306A0A43023B1343DA05400A4002C9
:100EF000D20D02433262F8229201306A1340B84A9E
:100F0000024013433362336A19433162326AB54B8C
:100F100013403362336AB44A134033620D92F3686C
:100F2000AC4A5B07FBD5072113698B4305390B439B
:100F30001361D3681B0603D5D3687E310B43D3609E
:100F400006F0F6FEA94804F05BFDFFF7F3FDF8207C
:100F500010A94002FFF796FDA54B109AA54C9A42A6
:100F600014D10025F823DB01E818800010A9FFF751
:100F700089FD109B6A0003936B469B890135A35240
:100F8000802DEFD1F9259C4F6D0216E0F82040022C
:100F9000FFF7A6FD0025994A6B009A5AE252E15AE2
:100FA000974BC918F823DB01E81880000135109130
:100FB000FFF73CFD802DEED1E4E710A92800FFF7F4
:100FC00061FD904B109AE9188F4B100E5854110C7C
:100FD0003970BA70110A8D4A043579700437954218
:100FE000EBD11A78FF2A10D1AA3A72211A701E3258
:100FF0005A700E3A9A70DA710022D9700439197158
:101000000D3959710C3199711A72FA2010A94002E8
:10101000FFF738FD2200109B80329BB210A97C485C
:101020001380FFF72FFDFFF795FDFF2362885B001C
:101030009A4202D9FE3BFF3B638023004C331A885F
:10104000052A01D900221A806388724A9BB2138054
:10105000638F1B0705D580216F4A890513680B43F1
:1010600013609721109B6D4A1B021B0A13601368C3
:1010700009065B189020C825136028226849FF30B4
:101080006D005300E75A8F4200D9E152E75A874278
:1010900000D8E552531C5B00E75ABC46604FBC4584
:1010A00000D9E152E75A874200D8E5520332402A7C
:1010B000E7D18025049BBF321869079B56499A6087
:1010C0000B68AD012B430B600392C30603D43F4B67
:1010D0001B69DBB203930C9B0A9A394F1A60039B7E
:1010E000FF2B01D100F002FE3C23039A1A4212D1D9
:1010F00008210720FFF77CFD8023802019000003D2
:10110000049A01339268034201D00A4300E08A4303
:10111000049CA260F4E77F23039A13401E2B21D185
:101120006B461B7B5BB2002B05DB05210220FFF722
:101130005FFD052104E000210220FFF759FD002199
:101140000320FFF755FD8023802019000003049A37
:1011500001339268034201D00A4300E08A43049CB1
:10116000A260F4E71D2B61D16B461B7B5BB2002BA9
:1011700006DB05210420FFF73BFD0521080005E003
:1011800000210420FFF734FD00210520FFF730FD8A
:101190008023802019000003049A013392680342DF
:1011A00040D00A433FE0C046555500000040005083
:1011B0004040005040550000C0400050CF5F00004C
:1011C00000410050FF0F0000FFFF00008040005072
:1011D0004000005000020050FFFFF7FFFC0100201C
:1011E000FFC1FFFFFFFFFBFFFFFFFEFF20A1070086
:1011F000A500FFFF20020020FD0600209CBC00008F
:101200000000FFFF000EFEFFFC06002018F20100A8
:10121000FC0F1000D006002068070020E401002029
:10122000B80B00008A43049CA260B5E71B2B21D1B8
:101230006B461B7B5BB2002B05DB05212020FFF7F3
:10124000D7FC052104E000212020FFF7D1FC00217C
:101250002120FFF7CDFC8023802019000003049A91
:1012600001339268034201D00A4300E08A43049CA0
:10127000A260F4E7172B21D16B461B7B5BB2002BDE
:1012800005DB05212220FFF7B3FC052104E0002146
:101290002220FFF7ADFC00212320FFF7A9FC8023CB
:1012A000802019000003049A01339268034201D0A0
:1012B0000A4300E08A43049CA260F4E76C23039A8B
:1012C0001340642B31D10121114007D16B461B7BA8
:1012D0005BB2002B00DB0F31242016E0039B9B0741
:1012E00008D46B461B7B00215BB2002B00DAFF2188
:1012F00040200AE0039BDB0609D46B461B7B0021E0
:101300005BB2002B00DB0F214120FFF771FC802234
:1013100080241000AA4B240301329968224201D094
:10132000014300E081439960F6E73F23039A9A4323
:1013300044D11024039B1C4063425C41039BA400E6
:101340009B0601D408231C430123039A1A4200D1AF
:101350001C430223039A1A4200D11C43052C00D9D6
:10136000002421002520FFF743FC8026002584422D
:1013700003D021002520FFF73BFC802149030023F7
:101380008C468F4A8021013309038D4F0B4202D0D6
:101390009168314301E09168B14391606345F1D1B7
:1013A0000135ADB2AC42E2D2BB68B343BB6084420C
:1013B000DCD021002520FFF71BFCD7E7039B5B0750
:1013C00000D481E2FEF766FF012264210320FEF7CC
:1013D0006BFF0320FFF70CF90320FFF7DBF8002376
:1013E000784A01210320FFF701F823004C331B88C2
:1013F000022B00D955E2E3889BB2039323899BB269
:10140000049363899BB20593A3899BB20693231D22
:10141000DB8F9BB20793A31DDD8F23004834083375
:10142000DE8F2388ADB29BB2B6B20893664BFF2124
:101430001869012301400B4000D086E0604A000695
:101440002DD48020916881439160039970380131D7
:1014500089B203910499013189B20491B968814339
:10146000B960B96810300143B960584916380B802B
:10147000039B58430B001C888442FCDB2024B86883
:10148000A043B860B868103C2043B86000200880D2
:101490000A210498414318888842FCDB33E04B065C
:1014A00035D4802193688B439360039B012B02D931
:1014B000013B9BB20393049B012B02D9013B9BB2DE
:1014C00004931021BB680A208B43BB60BB6849189A
:1014D0000B43BB6000233D490B80039B58430B002B
:1014E0001C888442FCDB2024B868A043B860B8683C
:1014F000103C2043B860002008800A210498414332
:1015000018888842FCDB1021BB688B43BB601369E1
:101510002B491B0719D480228B68022013438B6050
:101520000399FFF765FB039B834203D01900022058
:10153000FFF75EFB04990320FFF75AFB049B8342ED
:1015400003D019000320FFF753FB1F4BFF2118693D
:10155000022301400B4000D090E0194A000637D426
:10156000802091688446814391600599013189B258
:1015700005910699013189B206914021B8688843E6
:10158000B8606046B9680143B960104976380B808D
:10159000059B58430B001C888442FCDB8024B86800
:1015A000A043B860B868403C2043B8600020088081
:1015B0000A210698414318888842FCDB3CE0C0467B
:1015C000C04000508D770000804000501A0A002073
:1015D0004B0635D4802193688B439360059B012B88
:1015E00002D9013B9BB20593069B012B02D9013B1B
:1015F0009BB206934021BB680A208B43BB60BB684B
:1016000049180B43BB600023AC490B80059B584332
:101610000B001C888442FCDB8024B868A043B860BF
:10162000B868403C2043B860002008800A21069832
:10163000414318888842FCDB4021BB688B43BB6078
:1016400013699F491B0719D480228B680420134318
:101650008B600599FFF7CCFA059B834203D01900F4
:101660000420FFF7C5FA06990520FFF7C1FA069B8B
:10167000834203D019000520FFF7BAFA914B1020DE
:101680001969FF230B40184000D07FE08C4A0906FF
:101690002AD48021936801358B439360079B7F395F
:1016A00001339BB20793BB68ADB28B43BB60BB6891
:1016B00001310B43BB608149079B08800A305843C6
:1016C0000B001C888442FCDB0224B868A043B8608D
:1016D000B868013C2043B860002008800A216943B3
:1016E00018888842FCDB30E05B0632D480219368A6
:1016F0008B439360079B012B02D9013B9BB207935D
:10170000012D01D9013DADB20121BB680A208B43F7
:10171000BB60BB6849180B43BB60002367490B8063
:10172000079B58430B001C888442FCDB0224B868EA
:10173000A043B860B868013C2043B860002008802E
:101740000A21694318888842FCDB0121BB688B436E
:10175000BB6013695A491B0718D480228B6820206C
:1017600013438B600799FFF743FA079B834203D02B
:1017700019002020FFF73CFA29002120FFF738FA52
:10178000854203D029002120FFF732FA4D4BFF217B
:101790001869202301400B4000D047E6484A000664
:1017A0002AD48020916801368143916008997C3861
:1017B000013189B20891B968B6B28143B960B9689C
:1017C00004300143B9603D4902300B800B00704387
:1017D0001C888442FCDB0824B868A043B860B86861
:1017E000043C2043B860002008800A210898414347
:1017F00018888842FCDB30E04B0632D480219368A5
:101800008B439360012E01D9013EB6B2089B012B98
:1018100002D9013B9BB208930421BB680A208B4389
:10182000BB60BB6849180B43BB600023234970436E
:101830000B800B001C888442FCDB0824B868A043A2
:10184000B860B868043C2043B860002008800A21D2
:101850000898414318888842FCDB0421BB688B430D
:10186000BB60136916491B0700D5DFE580228B6832
:10187000222013438B603100FFF7BAF9864203D070
:1018800031002220FFF7B4F908992320FFF7B0F9BF
:10189000089B834200D1C9E519002320FFF7A8F96E
:1018A000C4E5082080220549054B0C88044202D07B
:1018B00000249C60F9E79A60F7E7C0461A0A002006
:1018C000C04000508040005023004C331B88BD4F67
:1018D000012B00D8F2E1FEF7DDFC01226421032098
:1018E000FEF7E2FC0320FEF783FE0320FEF752FE24
:1018F00001210023B44A0320FEF778FDB34AB44B1C
:101900000126136003F0D4FC002003F0E7FF16204B
:1019100003F014FB3223002112AD032013936970EE
:101920002E70159103F086FF2900032003F032FD8D
:101930003100032003F034FF3100032003F0D0FC1A
:10194000039B03229D080C231D40039B1340ED18AD
:101950000F235D406A43130028330493B340E45AD5
:101960009A4BA4B209939B4B03929C4206D89023B6
:10197000FF339C4203D8C824640000E0954C402605
:10198000BB682100B343BB600520FFF71BFA0323AC
:101990005D43ADB22B002833DBB206932B00293315
:1019A000DBB22A350793EBB2002508930A96022D85
:1019B00061D1894B1A88002A5DD0002287491A809C
:1019C000874A10880B88984227D2864B188813883C
:1019D000C3189BB2138010880B88984202D90B88D9
:1019E0009BB213807E4E0520318889B2FFF7EAF959
:1019F0007A4932880B889A420FD1049A7A4B500068
:101A0000C25A9446039A29325200D65AB44501D29A
:101A1000C35A00E0D35A9BB20B80714A6F491088B9
:101A20000B88984227D96F4B188813881B1A9BB2D2
:101A3000138010880B88984202D20B889BB21380C7
:101A4000674E0520318889B2FFF7BCF963493288B7
:101A50000B889A420FD1049A634B5000C25A9446A5
:101A6000039A29325200D65AB44501D2D35A00E023
:101A7000C35A9BB20B80099B1B691A0639D480227A
:101A8000BB689343BB60022D21D1059B56495E1C68
:101A9000039BB6B229335B005A5A9446049A52000B
:101AA000505A844503D95B5A505A181A02E0525AC8
:101AB000585A101A711C09F0FDFF4A4B80B2188069
:101AC000484B1A88002A0CD101321A800AE0414B97
:101AD0009C4201D00134A4B221000520FFF772F925
:101AE00000E0059600223C4B1A801A88012AFCD996
:101AF00037E00A9A134234D18022BB689343BB601B
:101B0000022D1ED1059B002B02D0013B9BB20593F9
:101B1000039B049A344929335B0052005E5A505AA1
:101B2000864203D95B5A505A181A02E0525A585A40
:101B3000101A059B591C09F0BDFF2A4B80B2188072
:101B400009E0C8235B009C4201D0013CA4B2210003
:101B50000520FFF737F900221F4B1A801A88012A47
:101B6000FCD93E69174A330700D520E780219368E6
:101B70000B439360012D39D0002D02D0022D65D08A
:101B80006FE021000698FEF7FBFF844203D021009E
:101B90000698FEF7F5FF039B134A29335B009C5A16
:101BA0000C4BA4B29C4206D89023FF339C4203D82E
:101BB000C824640000E0074C21000520FFF702F96B
:101BC000012567E0C04000508D7700008040005044
:101BD000FFF70000B80B00001A0A0020E4060020FE
:101BE00078040020340A00202002002021000798F9
:101BF000FEF7C6FF844203D021000798FEF7C0FF1E
:101C0000039A344B2A325200D25A039992B2059267
:101C1000049A31485200D25A293192B202804900C6
:101C2000CD5A0288954203D9CB5A0088181A02E08F
:101C30000288C85A101A059B0225591C09F03AFF60
:101C4000264B80B21880264B1C8023E0059908980B
:101C5000FEF796FF059B834203D019000898FEF714
:101C60008FFF049B1B4A5B009C5A1E4BA4B29C42F4
:101C700006D89023FF339C4203D8C824640000E0B8
:101C8000184C21000520FFF79DF821000520FFF7E3
:101C900099F800250022144B1A801A88092AFCD9C9
:101CA0000823F6B21E4202D13E69F6B2FAE70022DC
:101CB0000D4B1A801A88092AFCD978E608210020E1
:101CC0008023094A14880C4201D0B860FAE7BB604F
:101CD000F8E7C04620020020E4060020340A002075
:101CE00078040020B80B00001A0A0020079B0B9A0A
:101CF000A0241A600323032200930023110018007C
:101D000009F0D0FC8C22D54B520088331B8801216E
:101D1000DBB2002009F0BCFD0121D04BFA228A334E
:101D20001B880800DBB209F0EDFD0021CC4809F06A
:101D300015FD0021CB4809F037FD09F097FDCA4A8F
:101D4000CA4B1168E4050B4003210B431360C84ADA
:101D5000C84B116802200B40C02109010B431360DE
:101D60008022E36852021343E360E3680D9A042182
:101D700013408022E360B36852021343B360BE4B4A
:101D80009A680A439A609A6802439A609A68EE30A9
:101D900082439A60DA68D0388243DA60DA681D38A4
:101DA0000243DA60DA688A43DA60DA688A43DA6022
:101DB0001A6A03998A431A627269B04B13407361BD
:101DC000B5692D052B0F059303F0BEFD8022AC4DA8
:101DD00092052B68134380222B602B685205134316
:101DE0002B60059B591C09F0DBFDA64909F0D8FDC5
:101DF0002A68023883B2100C000418432860236B51
:101E0000A14A0025134008222363236B1420934327
:101E10002363236B9D4A13402363236B1340236387
:101E2000C3249B4BA4001B59039A93438022134362
:101E3000974A135103F082F8964B974A1D70974BBF
:101E400097491D701368DBB20B7096490B701F2306
:101E5000087803400B709449944B80200B60032357
:101E60000B7101234D718B71CD7113680A221343DD
:101E7000DBB240030B72FEF7F5FB01230EA98020B5
:101E80004B70052340030B708D70CD700D71FEF704
:101E90007BFD80202A0001214003FEF70BFD8022FC
:101EA000834B9201DA677A4B824A1B59290013400F
:101EB000774A0620135102F0CBFF0221032002F0E3
:101EC000AFFF0321080002F0ABFF0D2003F036F84E
:101ED0000E2003F033F80221774B2A00080002F0AD
:101EE000D3FF764B2A000121032002F0CDFFC02250
:101EF000C021674B92009B5809061B021B0A0B432B
:101F000063498B50FEF7C6F901226D492800FEF7A0
:101F1000CBF92800FEF76CFB2800FEF73BFB012203
:101F2000FA2110008900FEF7BFF90120FEF760FBDF
:101F30000120FEF72FFB01212B00624A0800FEF76B
:101F400055FAC222524B92009B585A4910200B401E
:101F5000C02109020B434E49404C8B500121B3680C
:101F60000343B360584B1D609A680A4380219A600E
:101F70001A68C9050A4380211A601A6849020A438F
:101F80001A601968514A11408022120511431960E4
:101F90001A6803998A4302431A60304B3A4A4C3319
:101FA0001B880B92394A0C92394A0392012B00D8B4
:101FB000E8E2260080363388454A9BB2138003F05E
:101FC00077F9152002F0BAFF01220CAB1A76322302
:101FD0002900139328000CAB5D76159503F02AFCBD
:101FE00012A9280003F0D6F90121280003F0D8FB3C
:101FF0000121280003F074F9FA22364B52001A80AE
:10200000012336881E40AE420BD02600523631885E
:10201000280089B2FEF7D6FE01222F4B1A703388B2
:1020200009E0250050352988300089B2FEF7CAFE44
:10203000294B1E702B88294A9BB21380284A210005
:102040001380220026005032523110880B88254D13
:102050005436984248D91388088847E02002002067
:102060001D7600004D7600003C000050FCFCFFFF98
:1020700030000050F3F3FFFF00000540FFFFFFFCBE
:102080002400054090D00300FFF7FFFFFFFBFFFF98
:1020900000E100E03D0A0020E4010020E001002012
:1020A000EA060020C10500200402002020A107004C
:1020B00004E100E0FF00FFFF295A00008D5F0000EF
:1020C00048E80100C963000000001140FFFFFFE77E
:1020D000E8010020B8040020E9060020E406002002
:1020E00078040020340A00200B8810883188181AE0
:1020F00080B2013109F0DEFC80B228802B88002BF1
:1021000001D101332B800221012003F093FB12A99E
:10211000012003F03FF90121080003F041FB0121F8
:10212000080003F0DDF82300022280331B88B04D45
:10213000260013420BD058363188012089B2FEF7B1
:1021400041FE0221AB4A13780B43137005E056366B
:102150003188012089B2FEF735FE3388A64A9BB24A
:102160002B8021001380220026005632583110881F
:102170000B885A36A14D984202D91388088801E08D
:102180000B8810883188181A80B2013109F092FC4E
:1021900080B228802B88002B01D101332B801620A0
:1021A00002F0CCFE0221080003F044FB12A9022039
:1021B00003F0F0F80121022003F0F2FA01210220DD
:1021C00003F08EF82300102280331B888C4D2600EC
:1021D00013420BD06A363188042089B2FEF7F2FD33
:1021E0001021844A13780B43137005E06836318858
:1021F000042089B2FEF7E6FD3388824A9BB22B8029
:10220000210013802200260068326A3110880B8872
:102210006C367D4D984202D91388088801E00B88FE
:1022200010883188181A80B2013109F043FC80B25D
:1022300028802B88002B01D101332B800221032021
:1022400003F0F8FA12A9032003F0A4F801210320F7
:1022500003F0A6FA0121032003F042F82300202214
:1022600080331B88694D260013420BD070363188AD
:10227000052089B2FEF7A6FD20215E4A13780B43A4
:10228000137005E06E363188052089B2FEF79AFD9D
:1022900033885F4A9BB22B802100138022002600E6
:1022A0006E32703110880B8872365A4D984202D9BE
:1022B0001388088801E00B8810883188181A80B2CA
:1022C000013109F0F7FB80B228802B88002B01D167
:1022D00001332B80172002F031FE0221042003F08D
:1022E000A9FA12A9042003F055F80121042003F0F3
:1022F00057FA0121042002F0F3FF23000422803367
:102300001B88454D260013420BD05E3631880220D3
:1023100089B2FEF757FD0421364A13780B43137038
:1023200005E05C363188022089B2FEF74BFD338828
:102330003A4A9BB22B8021001380220026005C3297
:102340005E3110880B886036354D984202D913886B
:10235000088801E00B8810883188181A80B2013192
:1023600009F0A8FB80B228802B88002B01D1013313
:102370002B800221052003F05DFA12A9052003F04D
:1023800009F80121052003F00BFA0121052002F0D4
:10239000A7FF2300082280331B88224D260013420A
:1023A0000BD064363188032089B2FEF70BFD08217B
:1023B000104A13780B43137005E06236318803200E
:1023C00089B2FEF7FFFC3388174A9BB22B802000AE
:1023D000138022002100623064320688138866313F
:1023E000124D9E4224D9230050331B88108821E0CF
:1023F0007A040020E9060020F6060020620700208B
:1024000000020020100200201008002058070020C1
:10241000020200207E04002098040020180A0020F8
:10242000B6040020660700209E040020B4040020AB
:10243000138800880988181A80B2013109F03AFB24
:1024400080B228802B88002B01D101332B801820EB
:1024500002F074FD0221062003F0ECF912A9062017
:1024600002F098FF0121062003F09AF901210620CD
:1024700002F036FF2300402280331B88C74D260020
:1024800013420BD076363188062089B2FEF79AFCCB
:102490004021C34A13780B43137005E0743631882A
:1024A000062089B2FEF78EFC3388BE4A9BB22B8091
:1024B00021001380220026007432763110880B88A8
:1024C0007836B94D984202D91388088801E00B8804
:1024D00010883188181A80B2013109F0EBFA80B205
:1024E00028802B88002B01D101332B80022107206B
:1024F00003F0A0F912A9072002F04CFF01210720E8
:1025000003F04EF90121072002F0EAFE2300803398
:102510001B88A64D26001B060CD57C36318807206B
:1025200089B2FEF74FFC80219D4A494213780B4344
:10253000137005E07A363188072089B2FEF742FC35
:1025400033889B4A9BB22B802100138022002500F8
:102550007A327C3110880B887E35964E984202D9AB
:102560001388088801E00B8810882988181A80B21F
:10257000013109F09FFA80B230803388002B01D1FD
:102580000133338023004C3318888B4D80B20528EB
:1025900034D809F0F1F928030D181818079B0A9A86
:1025A0001B681A431300079A1360FF23079A24E05D
:1025B0002B88824A01339BB213802B88804A0233D6
:1025C0009BB213801AE02B887C4A9BB213802B8825
:1025D0007B4A01339BB213805523089A1360099AF2
:1025E000153B13600AE05523089A1360099A153BBE
:1025F00013600023089A9360099A936003F048F9E6
:10260000704B714A1B68714B1B6800231360536049
:102610009360D360136153619361D3616C4A13700B
:1026200023004C331A88012A02D01B88032B05D1C2
:102630008021684A490313680B4313603F237021CC
:102640002A881340803B644ADBB213702B889B09B5
:102650000B40537053784B4053705378803BDBB240
:102660005370A38FDB0705D580215A4A890513686B
:102670000B4313608023594A9B01136000230426F7
:10268000079380330393564C236833422DD0FEF7D3
:1026900069FAFEF74FFAF9204002FEF721FAF92312
:1026A000504D5B020593059B4F4A05989B184F4A76
:1026B000D35C1A062B781B04D3186A7812029B1875
:1026C000AA7804359B1819000393FEF7AFF9059B10
:1026D000043305931A1E464B9A42E4D1FEF73AFAA8
:1026E00003F0D6F82368B34323603A4C23689B0277
:1026F00008D423689B0305D48022049B9B689343E2
:10270000049A93603B4B3C4D1A88254BD2B21B7800
:102710009A4200D1D1E080222978D204002971D1D7
:102720002068104000D0EBE00A232B7005252368B9
:102730001A43324B22601978C9B24A1CD2B21A70BD
:102740002F4A55541978C9B24D1CEDB21D7056541C
:102750001978C9B24D1CEDB21D7050541978C9B228
:10276000481CC0B218701A4805918446614600782A
:10277000C0B2451CEDB20D70059950541878C0B226
:10278000411CC9B219708E2111541978C9B2481C64
:10279000C0B21870012353548AE0C0468004002060
:1027A000E9060020F4060020300A0020FA06002086
:1027B0007C040020160A0020D00600202C0A0020ED
:1027C000F806002010400050EC000020504000505F
:1027D000E8060020680700205F04002000E100E018
:1027E000280A0020FD060020000EFEFFFC06002047
:1027F00018F20100E80100206C07002016020020FA
:10280000CF050020256815407AD121689BB20A4384
:102810002260C84A1380FEF7A5F9FEF78BF9FA206B
:102820004002FEF75DF9FA20C24B4002198889B2D6
:10283000FEF7FCF8FEF78EF903F02AF80520BE4BF0
:102840001978C9B24A1CD2B21A70BC4A50541978CD
:10285000C9B2481CC0B2187056541978C9B2481C85
:10286000C0B2187055541978C9B2481CC0B218705B
:10287000B348059184460078C1B208910131C9B2CC
:1028800008006146087005996846029120214018A9
:102890000078029950541878C0B2411CC9B219701E
:1028A0008E2111541978C9B2481CC0B21870555401
:1028B0002268A44B1340236022E0A34B1B78DBB2B9
:1028C0000593032B15D1A14B1A78A14B1B789A4283
:1028D0000DD1A04B1B88002B0BD123689B0108D482
:1028E00005F0B2FA6A469B4B928A1A8001E005F025
:1028F000ABFA2B78002B03D02B78013BDBB22B708B
:102900000122954B954D1868104000D146E16A8F21
:10291000196892B2090702D41B681B022FD4082041
:102920008D490B68034200D1FDE08D4C237864781B
:1029300083401B190393039C8A4B9C4207D16B8FE6
:10294000034204D080200B68800503430B6093068C
:1029500000D5C9E0702382494A781A40824B12029E
:102960001A601A6892091A603F22087819680240B2
:102970005218E0211A601A6849004A401A60764CE1
:1029800023689B021AD5774B039A9A4216D0764B4E
:10299000764A1B6800209BB21380118889B2FEF72B
:1029A00027F98021704B1B689BB26B802268704BAB
:1029B0001340704A236093688B4393606B4B6A4A61
:1029C0001B8811685B1A59425941CBB205932B0001
:1029D0004C331B88012B0BD9674B1988136899421C
:1029E00001D102230593654B19881368994204D0DD
:1029F000059B002B00D177E001E0032305930F2115
:102A0000574A93788B43E02B25D19178D43B0B40E8
:102A10000C2B20D19178093BD2780B401B029B18DC
:102A20000893062B17D005244D4B202219796B46AD
:102A30009B181878FEF7DCF8494B1B7998420AD0AE
:102A4000013CE4B2002CEFD14D4B984203D1FEF78C
:102A500089F802F02BFF434B039A9A4244D0072394
:102A60003F4A3E4C50780599184001383A4B0628A9
:102A700001D800F0D1FF022901D101F063F8032948
:102A800001D000F0D2FF23003E4D3F4A2E706A3342
:102A900019881288914201D101F09EF81B883A4AA8
:102AA0009BB213801022234B40201B888034134399
:102AB000204A1380118889B2FEF762F81D4B1B88EB
:102AC0009BB22380314B1E7000236B700533AB70BB
:102AD0002D4B18882E4B80B219882E4B89B21A883C
:102AE00092B2FEF7A3F9E8701B4B1A68D2051AD50B
:102AF0004821204A91600022BA601B681B0510D54E
:102B0000174B1A7892070ED15A78452A01D802F04D
:102B10007FF85A788A2A06D95A78A32A03D802F06D
:102B200077F8FEF711F90C4A1B4B11680B40136044
:102B3000A9E5C046E801002016020020CF050020CC
:102B4000E8060020FFFFFFFB3D0A00203E0A0020B0
:102B5000320A0020840400206807002020020020A0
:102B6000610400200FBF0000FC010020D0060020FF
:102B7000FFFFDFFFC04000502C0A0020F8060020B5
:102B8000FFFF0000C905002000020020A104002072
:102B90001002002010080020FCFFFEFF079A013AF7
:102BA000D2B207922A004C32118889B2012901D190
:102BB00000F0BFFB002902D0032900D063E5079B8A
:102BC000002B00D05FE5AB4B1C692B004C331B88FE
:102BD000002B00D080E08022630063400393134207
:102BE00014D0A54B620603D401219A680A4302E07F
:102BF00001219A688A4301219A60A04A13688B4395
:102C00001360FC23069A1A40069225E02B0001214E
:102C100084331B880B421FD00120994B99491B8894
:102C2000013B9B009BB20B8094490B6803430B60F4
:102C3000954B1B685B030FD5069B0100034206D131
:102C40000798144201D10799080008F0B5FC032346
:102C5000069A1343DBB206932021039B0B4213D049
:102C6000854A1E39E30602D493680B4301E093685A
:102C70008B4302219360814A13688B431360F323D3
:102C8000069A1A40069270E10222804B84331B8818
:102C9000134200D169E17A4B7A481B889340033B89
:102CA0009BB20380754803681A43774B02601B6828
:102CB0005B0300D459E1069B334207D12140012038
:102CC000002901D00121080008F076FC0C23069AA7
:102CD0001343DBB2069348E16D4A1378002B00D012
:102CE00043E16C4B610632D5C82111701978079AFF
:102CF000012902D001221A700122674B674D198801
:102D00002B8899422BD140205C490B6803430B6010
:102D10005E4963488C46012103780B4207D0614627
:102D20005031098889B2298001218B4306E0614630
:102D30005231098889B2298001210B430370504B1D
:102D400050491B88013B9B009BB20B8007E0197820
:102D5000079A002903D06A46127F1A7001224A4B53
:102D60004C4D1968490309D51B68DB0206D5002ABA
:102D700004D029780020C9B208F038FB8023234012
:102D800032D0C822424B1A706A780023012A02D03E
:102D900001336B700123434A1188434A94461288D9
:102DA000914226D18020022534490A6802430A60F4
:102DB0003B4A364912782A4206D060465631098885
:102DC000AA4389B2018005E06046583109882A4348
:102DD00089B2018032490A70294A2A491288920030
:102DE000033A92B20A8004E06A78002A01D06B703C
:102DF0000123254A274D1168490309D51268D202DB
:102E000006D5002B04D069780120C9B208F0EEFA8B
:102E1000102323404ED0C8221D4B1A70AA780023DD
:102E2000012A02D00133AB700123204A204D1188C2
:102E30002A88914243D18020104940000A68024309
:102E400017480A6002781149324205D05C3109887E
:102E5000B24389B2298004E05E310988324389B2E5
:102E600029800270064A074912889200023A92B2FB
:102E70000A8024E04040005080400050200A00209A
:102E8000D0060020860400206807002020020020D1
:102E9000A00400201702002078040020E40600208F
:102EA000E9060020F60600207A040020180A002017
:102EB00098040020AA78002A01D0AB700123B44AFC
:102EC000B44D1168490309D51268D20206D5002B0A
:102ED00004D0A9780220C9B208F088FA20210C4059
:102EE0002FD0C822AC4B00241A70EB78012B02D0F3
:102EF00001230134EB70A94BA94D1A882B889A4203
:102F000024D180210820A74A890013680B43A649D1
:102F100013600B78A54A034205D0623212888343BE
:102F200092B22A8004E064321288034392B22A806B
:102F30000B709F4B9F4A1B889B00023B9BB21380E8
:102F400004E0EB78002B01D0EC700124904B1A6860
:102F500052030AD51B68DB0207D5002C05D08D4B28
:102F60000320D978C9B208F041FA934B1B69039347
:102F70008E4B1A004C321288002A00D080E080214B
:102F8000039A540054400C4213D08C4B20200A4228
:102F900002D19A68024301E09A68824308219A604C
:102FA000804A13688B4313603F23069A1A400692A7
:102FB00024E0082284331B8813421FD07C4B7D48B9
:102FC0001B889B00013B9BB20380764803681A4331
:102FD0006F4B02601B685B0310D5C023069A1A4230
:102FE00006D1039B194000D00121032008F0E4FA28
:102FF0004023069A5B421343DBB2069320210C4226
:1030000014D0039A6D4B10200A4202D19A680243F1
:1030100001E09A6882439A60624A1368B34313607E
:10302000CF23069A1A400692FFF72DFB5F4B84339D
:103030001B88334201D1FFF726FB5D4B5D4A1B889D
:103040009B00023B9BB21380564A136833431360C4
:103050004F4B1B685B0301D4FFF715FB3023069A27
:103060001A4206D1039B194000D00121032008F029
:10307000A3FA3023069A1343DBB20693FFF703FB50
:1030800045480378D9B2002901D0FFF7FCFA202384
:10309000039A13403F4A30D0C823037010790B00C5
:1030A000012802D0013313710123454A454D11888F
:1030B0002A88914226D1802010243A49C0000A680B
:1030C000024339480A6002783849224205D0683103
:1030D0000988A24389B2298004E06A310988224321
:1030E00089B229800270324A3249128892B20A802B
:1030F0000A88920092B20A8004E01179002901D076
:1031000013710123224A234C1168490309D512681F
:10311000D20206D5002B04D021790420C9B208F0D0
:1031200065F91023039A134052D0C8221A4B1A7023
:1031300062790023012A02D0013363710123224AFC
:10314000224D11882A88914247D180202024154998
:1031500000010A68024314480A60027813492242B7
:1031600005D06E310988A24389B2298004E070310C
:103170000988224389B2298002700D4A0D491288BC
:1031800092B20A800A889200013292B20A8024E048
:103190006807002017020020A00400209E040020E1
:1031A00066070020200A0020E906002020020020F7
:1031B000D0060020860400200040005080400050CF
:1031C0001002002000020020020200205807002008
:1031D0006279002A01D063710123B74AB74C1168A4
:1031E000490309D51268D20206D5002B04D06179B3
:1031F0000520C9B208F0FAF88023039A134032D0B0
:10320000C822AF4B1A70A2790023012A02D00133E1
:10321000A3710123AB4AAC4D11882A88914227D172
:1032200080204024A94940010A680243A8480A6056
:103230000278A849224205D074310988A24389B294
:10324000298004E076310988224389B229800270FE
:10325000A14AA249128892B20A800A8892000232D8
:1032600092B20A8004E0A279002A01D0A37101235E
:10327000914A924C1168490309D51268D20206D5C9
:10328000002B04D0A1790620C9B208F0AFF8402382
:10329000039A134035D0C822894B1A70E279002373
:1032A000012A02D00133E37101238D4A8D4C11882C
:1032B000228891422AD18020844980010A680243F1
:1032C00083480A600178834A4DB2002D06DA7A32CB
:1032D000128892B222807F22114006E07C3212884E
:1032E00092B222808022524211437B4A017012889E
:1032F0007A4992B20A800A889200033292B20A8016
:1033000004E0E279002A01D0E37101236A4A1168DE
:10331000490301D4FFF7B7F91268D20201D4FFF7CD
:10332000B2F9002B01D1FFF7AEF9644BD979C9B2DC
:103330006DE380246C4AE402126903920A4055D17D
:103340001868204205D01B68DB0202D5100008F087
:103350004DF8EB88002B0FD02022BB6801211343CE
:10336000BB606423EA885343604A9BB21380604A7F
:1033700013780B4313701AE05C490B88002B16D1AD
:1033800001205B4B1A78024206D01A7882431A70E9
:103390002022BB68934306E001201A7802431A708A
:1033A0002022BB681343BB60FA239B000B800121E2
:1033B000504A13780B4313702B004A331B880B427F
:1033C00007D0137849188B4313701022BB689343BE
:1033D000BB6040213D4A13680B4313603E4B3F4A9C
:1033E0001B88013B9B009BB2138008E01A682242B5
:1033F00005D01B68DB0202D5010007F0F7FF802231
:1034000003992D4BD202890700D577E01968114244
:1034100006D01B68DB0203D50121080007F0E6FF98
:103420002B89002B0FD01022BB6802211343BB60F5
:1034300064232A895343304A9BB213802C4A137861
:103440000B43137019E02C490B88002B15D1022077
:10345000274B1A78024206D01A7882431A7010223B
:10346000BB68934305E01A7802431A701022BB68C8
:103470001343BB60FA239B000B8002211D4A137883
:103480000B4313702B004A331B8801390B4206D0C3
:1034900013788B4313702022BB689343BB60402199
:1034A0000A4A13680B4313600B4B0C4A1B88013B01
:1034B0009B009BB213802BE06807002017020020BE
:1034C000A0040020F406002080040020200A002030
:1034D000E906002020020020D006002086040020FB
:1034E0007C040020FA060020804000509A0400204E
:1034F0006007002090040020820400201968114217
:1035000006D01B68DB0203D50021012007F06EFF07
:1035100080220399C64BD202C90652D419681142BF
:1035200006D01B68DB0203D50121022007F05EFFF5
:103530006B89002B0ED08022BB681343BB606423D1
:103540006A895343BB4A9BB21380BB4A1378334307
:10355000137018E0B7490B88002B14D1B64B1A78BA
:10356000324206D01A78B2431A708022BB68934365
:1035700005E01A7832431A708022BB681343BB609F
:10358000FA239B000B80AD4A1378334313702B0052
:103590004A331B889B0707D5082113788B43137088
:1035A0004022BB689343BB608021A54A13680B434C
:1035B0001360A44BA44A1B889B00033B9BB213805F
:1035C00009E01968114206D01B68DB0203D500210F
:1035D000022007F00BFF80220399954BD202890647
:1035E00054D41968114206D01B68DB0203D50121AF
:1035F000032007F0FBFEAB89002B0FD04022BB68F5
:1036000008211343BB606423AA8953438F4A9BB2AA
:103610001380894A13780B43137019E08B490B8888
:10362000002B15D10820844B1A78024206D01A7854
:1036300082431A704022BB68934305E01A78024324
:103640001A704022BB681343BB60FA239B000B80B7
:1036500008217A4A13780B4313702B004A331B88D6
:103660009B0706D51378B34313708022BB6893433E
:10367000BB608021724A13680B431360714B724A1E
:103680001B889B00033B9BB2138009E01968114221
:1036900006D01B68DB0203D50021032007F0A6FE3D
:1036A00080220399624BD202314257D119681142EC
:1036B00006D01B68DB0203D50121042007F096FE2B
:1036C0002A1DD38F002B0FD00221BB680B43BB6098
:1036D0006423D28F0E3153435D4A9BB21380564A06
:1036E00013780B43137019E059490B88002B15D13F
:1036F0001020514B1A78024206D01A7882431A7071
:103700000222BB68934305E01A7802431A70022232
:10371000BB681343BB60FA239B000B801021474A10
:1037200013780B4313702B004A331B88334207D0A6
:10373000137849188B4313700122BB689343BB6015
:1037400080213F4A490013680B4313603D4B3E4ABA
:103750001B889B00023B9BB2138009E01968114251
:1037600006D01B68DB0203D50021042007F03EFED3
:10377000802203992E4BD20209076DD41968114299
:1037800006D01B68DB0203D50121052007F02EFEC1
:10379000AA1DD38F002B0FD00121BB680B43BB6048
:1037A0006423D28F1F3153432A4A9BB21380224A8B
:1037B00013780B4313701AE0254B1B88002B16D18E
:1037C00020211D4B1A780A4206D01A788A431A70B3
:1037D0000122BB68934305E01A780A431A7001225C
:1037E000BB681343FA22BB601A4B92001A80202157
:1037F000124A13780B4313702B004A331B88334251
:1038000007D0137810398B4313700222BB6893439F
:10381000BB6080210A4A490013680B431360094BBF
:10382000094A1B889B00023B9BB213801EE0C046E6
:10383000680700208A040020600700209004002010
:10384000200A0020D006002086040020E606002082
:10385000EC060020120800201968114206D01B68EF
:10386000DB0203D50021052007F0C0FD802203996B
:10387000C74BD202490657D41968114206D01B68BB
:10388000DB0203D50121062007F0B0FD2A00083233
:10389000D38F002B0FD00821BB680B43BB60642380
:1038A000D28F38315343BB4A9BB21380BA4A137844
:1038B0000B43137019E0B7490B88002B15D140203A
:1038C000B54B1A78024206D01A7882431A70082241
:1038D000BB68934305E01A7802431A700822BB685C
:1038E0001343BB60FA239B000B804021AB4A137843
:1038F0000B4313702B004A331B881B0706D57F230D
:1039000011780B401370BB68B343BB608021A44A9D
:10391000890013680B431360A24BA34A1B889B00CA
:10392000013B9BB2138009E01968114206D01B6865
:10393000DB0203D50021062007F058FD8022039901
:10394000934BD202090657D41968114206D01B685E
:10395000DB0203D50121072007F048FD2A00483289
:103960001388002B0ED0BB683343BB6064231288DE
:1039700053438E4A9BB213808023874A11780B43AE
:10398000137018E089490B88002B14D1824B1A78E8
:10399000187852B2002A05DA7F2202401A70BB68FA
:1039A000B34304E0802202431A70BB683343BB6018
:1039B000FA239B000B808023784A11780B43137005
:1039C0002B0008214A331B880B4206D04020137875
:1039D00083431370BB688B43BB608021704A8900AE
:1039E00013680B4313606F4B6F4A1B889B00013BAE
:1039F0009BB21380FEF747FE1968114201D1FEF712
:103A000042FE1B68DB0201D4FEF73DFE00210720C9
:103A100007F0ECFCFEF737FE07F0B8FFF7002B02CB
:103A20003A0388045305AE06AB07E18800295FD04E
:103A300053781B0703D52022BB681343BB60564B4A
:103A40001A7801231A402CD10121594B1E705A704B
:103A5000524A12780A4207D05A783F310A435A70C4
:103A60000222544B1A700CE005229A70524AD188F7
:103A70003F2902D8D288D2B200E03F22DA704D4B03
:103A80001E702300012284331B88134204D020219E
:103A9000474A53780B4353703D4A484B11680B40DB
:103AA000136001224A342388134208D00221BB68E4
:103AB0000F329343394ABB6013788B4313706423EE
:103AC0000121EA8853433E4A9BB21380324A13785D
:103AD0000B4313703B4B5B781B072ED52B004C33ED
:103AE0001B88002B29D1384A93680B43936024E04C
:103AF0002F4A3249167018680140196030490B8806
:103B0000002B1AD10124244B1878204206D01878B3
:103B1000A0431870B8681F34A04306E00124187849
:103B200020431870B8681F342043B8601878032306
:103B300003405370FA239B000B80184A012113782D
:103B400000F0AAFF1A4B214A1E7023005233188836
:103B50001188884213D01B884C349BB21380238871
:103B6000042B07D12022BB689343BB60BB68103A8B
:103B70009343BB600122164C23881343F2E0154B9C
:103B800010881988884200D014E140230FE1C04614
:103B9000680700205E0700206007002090040020D6
:103BA000200A0020D00600208604002014070020F0
:103BB000C9050020A104002020020020FFFFFFBF54
:103BC0009A0400206104002080400050E406002098
:103BD000E801002078040020BC4B1988BC4B1A88EF
:103BE000914203D140236B7001F00DF805222A7039
:103BF000B64A10881988B74B80B21A8889B292B237
:103C0000FDF714F9687000F0FEFF022900D18DE085
:103C1000032900D1F3E0218900295ED053781B07E6
:103C200003D51022BB681343BB600221AA4B1B784B
:103C30000B422AD10122A94B1E705A70A84A127851
:103C40000A4206D040205A7802435A70A54B197098
:103C50000BE005229A7022893F2A02D82289D2B22B
:103C600000E03F22DA709F4B1E7023000122843354
:103C70001B88134204D02021984A53780B43537079
:103C8000994A9A4B11680B40136001224A342388E9
:103C9000134208D00121BB681F329343904ABB6096
:103CA00013788B431370642302212A895343904A6B
:103CB0009BB21380884A13780B4313708D4B5B784B
:103CC0001B072ED52B004C331B88002B29D18A4A89
:103CD000013993688B43936023E0804A83491670CF
:103CE00018680140196082490B88002B19D1022401
:103CF000794B1878204206D01878A0431870B8681D
:103D00000E34A04305E01878204310241870B868DA
:103D10002043B8601878032303405370FA239B00B4
:103D20000B806F4A0221137800F0B6FE6B4B734A8A
:103D30001E702300503318881188884231D01B88A8
:103D40004C349BB213802388042B07D12022BB68FC
:103D50009343BB60BB68103A9343BB600122684C3D
:103D60002388934323802188402089B2FCF708FFF1
:103D70002A00238880329BB213805A4B574C1E7006
:103D8000002363700533A3705C4B18885D4B80B2D1
:103D900019885D4B89B21A8892B2FDF747F8E07036
:103DA00019E0584B10881988884203D141234B4AA7
:103DB00053700DE005214948017010881988524B55
:103DC00080B21A8889B292B2FDF730F8434B58702E
:103DD0000222444B1A704D4B4C331B88052B01D0EB
:103DE000FEF782FE20213D4A53780B435370484A28
:103DF000484B11680B401360474B00F0B4FE2300A2
:103E0000324D683319882A88914221D010221B88AC
:103E100040209BB22B803A4B80341B889343384A16
:103E20001380118889B2FCF7ABFE354B1B889BB21F
:103E300023802C4B294C1E70002363700533A37024
:103E4000234B2888198880B289B2224B00F0BFFE2C
:103E50001F4B29881A88214C914201D100F0C4FEE1
:103E6000052222702888198880B289B2194B00F087
:103E7000C5FE022900D1B2E0032900D1F0E061893A
:103E8000002900D183E053781B0703D58022BB684B
:103E90001343BB60104B1A78324052D10F4B1E7047
:103EA0005A700F4A1278324207D040215A780A439A
:103EB0005A7002220B4B1A7034E005229A70628904
:103EC0003F2A2BD86289D2B229E0C04600020020E6
:103ED000100200201008002060070020C905002003
:103EE00090040020A104002068070020FFFFFFBF0E
:103EF000820400206104002080400050E40600207D
:103F0000E801002078040020340A0020200200206C
:103F1000200A0020FFFEFFFF404000503F22DA70E1
:103F2000C44B1E70230084331B889B0704D52021BB
:103F3000C14A53780B435370C04AC14B11680B40C0
:103F400013604A3423889B0708D50821BD4A13789B
:103F50008B4313704022BB689343BB6064236A8920
:103F60005343B94A9BB21380B84A13783343137052
:103F7000B74B5B781B072DD52B004C331B88002BD0
:103F800028D10221B34A93680B43936022E0AA4AE6
:103F9000AB49167018680140AB4819600388002BC4
:103FA00018D1AA4B1978314206D080241978B14330
:103FB0001970B968A14305E080241978314319705C
:103FC000B9682143B960FA21890001801B781B0779
:103FD0009B0F53709B4A1378334300F05EFD230020
:103FE0009D4A583318881188884220D01B884C3449
:103FF0009BB213802388042B07D18022BB68934394
:10400000BB60BB68403A9343BB600222894B934C30
:104010001E702388402013432380218889B2FCF737
:10402000AFFD2A00238880329BB21380E6E08C4BE0
:1040300010881988804C884202D1402363700BE0BD
:104040000521217010881988864B80B21A8889B2A0
:1040500092B2FCF7EBFE60700223764A137018E10F
:104060002300814D703319882A88914207D020227D
:104070001B889BB22B80794B1B8813432AE17B4B17
:1040800029881A886C4C914200D046E100F06FFC00
:10409000022900D18BE0032900D10DE1A18900297B
:1040A0005CD053781B0703D54022BB681343BB6029
:1040B0000822664B1B7813422AD101215E4B1E70E9
:1040C000597060490978114207D040215A780A4353
:1040D0005A700222574B1A700BE005229A70A2897F
:1040E0003F2A02D8A289D2B200E03F22DA70514BB7
:1040F0001E70230084331B889B0704D520214E4A61
:1041000053780B4353704D4A4D4B11680B4013606D
:104110004A3423889B0707D54A4A1378B343137060
:104120008022BB689343BB606423AA8947495343F9
:104130004F4A9BB2138008220B7813430B70444BF9
:104140005B7813422ED02B004C331B88002B29D1D7
:104150000221404A93688B43936023E0364A3849F2
:10416000167018680140196041490B88002B19D15D
:104170000824364B1878204206D01878A0431870CF
:10418000B8683834A04305E01878204340241870FC
:10419000B8682043B8601B781B079B0F5370FA2345
:1041A0009B000B80274A0821137800F075FC230040
:1041B000294A563318881188884231D01B884C34DC
:1041C0009BB213802388042B07D18022BB689343C2
:1041D000BB60BB68403A9343BB6002221F4C402047
:1041E000238893432380218889B2FCF7C9FC2A00E5
:1041F000238880329BB213800E4B1E7000230E4C1E
:1042000063700533A370144B1888154B80B219885E
:10421000144B89B21A8892B2FCF708FEE07038E0BD
:104220000F4B10881988044C884223D141236370B6
:104230002CE0C046A1040020C9050020680700202A
:10424000FFFFFFBF900400208A04002060070020C9
:1042500061040020804000507A040020E801002022
:10426000F606002062070020580700200202002006
:10427000E60600200521217010881988C64B80B2FF
:104280001A8889B292B2FCF7D1FD60700222C34B4A
:104290001A70C34B4C331B88052B01D0FEF724FC4E
:1042A0002021C04A53780B435370BF4ABF4B11685B
:1042B0000B401360BE4B27E22300BE4D6E331988BE
:1042C0002A88914221D020221B889BB22B80BA4B96
:1042D0001B889343B84A402013801188803489B2E8
:1042E000FCF74EFCB44B1B889BB22380AB4BAD4C10
:1042F0001E70002363700533A370B04B28881988A3
:1043000080B289B2AE4B00F062FCAC4B29881A88AF
:10431000A44C914201D100F067FC0522227028884C
:10432000198880B289B2A64B00F068FC022900D13E
:104330008DE0032900D1ADE0211DC98F00295ED099
:1043400053781B0703D50222BB681343BB601021BF
:104350009C4B1A780A402BD1924B1E705A709A4A85
:1043600012780A4207D05A7830310A435A70022232
:104370008A4B1A700DE005229A70894A0432D18F57
:104380003F2902D8D28FD2B200E03F22DA70834BAD
:104390001E70230084331B88334204D02021814ABD
:1043A00053780B435370894A894B11680B40136053
:1043B0004A342388334208D02021834A13788B4320
:1043C00013700122BB689343BB602B1DDA8F6423FB
:1043D000102153437F4A9BB213807A4B1A780A43C9
:1043E0001A707D4B5B781B072DD52B004C331B8837
:1043F000002B28D1794A93680B43936023E0694AE4
:104400007349167018680140196072490B88002BB7
:1044100019D110246B4B1878204206D01878A0438D
:104420001870B8680E3CA04305E0187820430224B9
:104430001870B8682043B8601B789B069B0F5370B8
:10444000FA239B000B80604A1021137824E3230099
:10445000634A5E3318881188884212D01B884C3416
:104460009BB213802388042B07D1BB68059A934322
:104470000122BB60BB689343BB604F4C238833432E
:10448000F9E0584B10881988464C884200D01AE150
:10449000402316E12300544D763319882A8891422F
:1044A00007D040201B889BB22B80434B1B880343C3
:1044B0003AE14E4B29881A883A4C914200D053E198
:1044C00055E2022900D1BDE0032900D11EE1A11D62
:1044D000C98F002900D18DE053781B0703D5012235
:1044E000BB681343BB602022364B1B7813422BD191
:1044F00001212C4B1E70597033490978114207D0A5
:1045000040215A780A435A700222244B1A700CE058
:1045100005229A70A21DD18F3F2902D8D28FD2B224
:1045200000E03F22DA701D4B1E70230084331B888D
:10453000334204D020211B4A53780B435370234A43
:10454000234B11680B4013604A342388334208D050
:1045500002221021BB6893431B4ABB6013788B4334
:104560001370AB1DDA8F642320215343204A9BB282
:104570001380144A13780B431370174B5B781B0797
:104580005CD52B004C331B88002B57D1134A1039B4
:1045900093688B43936051E062070020A1040020E0
:1045A00020020020C9050020200A0020FFFDFFFF97
:1045B0004040005058070020E8010020020200207F
:1045C0007E0400206007002090040020680700207F
:1045D000FFFFFFBFEC060020610400208040005078
:1045E00098040020180A002080040020F40600200F
:1045F00012080020C24AC3491670186801401960A9
:10460000C1490B88002B19D12024C04B18782042B7
:1046100006D01878A0431870B8681F3CA04305E086
:104620001878204301241870B8682043B8601B78BC
:104630009B069B0F5370FA239B000B80B44A2021EA
:10464000137829E22300B34A5C3318881188884222
:1046500030D01B884C349BB213802388042B07D1A5
:10466000BB68059A93430122BB60BB689343BB6060
:10467000A94C2388B34323802188402089B2FCF7CA
:104680007FFA2A00238880329BB21380A34B9C4C74
:104690001E70002363700533A3709E4B1888A04BD7
:1046A00080B219889F4B89B21A8892B2FCF7BEFB80
:1046B000E07017E09A4B10881988914C884202D11B
:1046C000412363700BE00521217010881988954BF8
:1046D00080B21A8889B292B2FCF7A8FB60700222FD
:1046E0008E4B1A70904B4C331B88052B01D0FEF774
:1046F000FBF92021824A53780B4353708B4A0C9963
:1047000013680B4013608A4B8A4A2DE223008A4DBE
:10471000743319882A8891421FD040201B889BB28D
:104720002B807D4B1B8883437B4A80341380118808
:1047300089B2FCF725FA784B1B889BB22380774B14
:104740006F4C1E70002363700533A3707B4B288869
:10475000198880B289B27A4B39E2784B29881A8855
:10476000674C914200D13FE20522227028881988C7
:1047700080B289B2724B41E2022900D18DE0032957
:1047800000D1AEE021000831C98F00295ED05378F6
:104790000822134202D0BB681343BB6040215B4B2D
:1047A0001A780A402AD1564B1E705A70584A12780D
:1047B0000A4206D05A780A435A700222574B1A709E
:1047C0000DE005229A70584A0832D18F3F2902D84D
:1047D000D28FD2B200E03F22DA70504B1E7023001D
:1047E00084331B881B0704D52021454A53780B438B
:1047F0005370544A434B11680B4013604A3423886A
:104800001B0707D57F23424A11780B401370BB6802
:10481000B343BB602B000833DA8F6423402153433A
:10482000494A9BB21380394A13780B431370474BA4
:104830005B781B072DD52B004C331B88002B28D110
:10484000434A203993680B43936022E02C4A2D4958
:1048500016701868014019603B490B88002B18D16D
:1048600040242A4B1878204206D01878A0431870AC
:10487000B868383CA04305E0187820430824187035
:10488000B8682043B8601B789B095370FA239B00DB
:104890000B801F4A40211378FEE023002D4A643329
:1048A00018881188884213D01B884C349BB213801F
:1048B00023889BB2042B06D10821BA688A43BA60C8
:1048C000BA689A43BA600822134C2388134301E163
:1048D000214B108819880A4C884200D022E14023DD
:1048E0001EE123001D4D7C3319882A88914237D060
:1048F00080221B889BB22B80074B1B8813434DE102
:10490000C9050020FFFFFFBF12080020600700203C
:104910009004002098040020E8010020A104002059
:10492000180A0020B604002020020020200A0020DF
:1049300000400050FFF0000080040020F40600203A
:10494000300A0020680700205E0700206104002074
:1049500080400050660700209E040020FA060020D8
:10496000CC4B29881A88CC4C914200D03FE140239F
:104970003BE1022900D193E0032900D100E12100AD
:1049800048310988002961D053781B0702D5BB68DC
:104990003343BB60C14B1B785BB2002B2DDB012284
:1049A000BD4B1E705A70BE4A127852B2002A07DA06
:1049B00040215A780A435A700222BA4B1A700DE00D
:1049C00005229A702200483211883F2902D81288A5
:1049D000D2B200E03F22DA70B24B1E702300843363
:1049E0001B881B0704D52021AB4A53780B43537017
:1049F000AD4AAE4B11680B40136008224A3423883D
:104A0000134207D04020A6490B7883430B70BB6844
:104A10009343BB602B0048331A8864235343A44A52
:104A20009BB2138080239D4A11780B431370A14BD6
:104A30005B781B072DD52B004C331B88002B28D10E
:104A400020219D4A93688B43936022E0924A9749C4
:104A50001670186801401960954B1B88002B18D1FF
:104A60008E4B1978187849B2002905DA7F21014068
:104A70001970B968B14304E0802101431970B96825
:104A80003143B9601B789B095370FA22884B92001E
:104A90001A808023824A11780B431370FEF724F8A2
:104AA0002300864A623318881188884231D01B88D7
:104AB0004C349BB2138023889BB2042B06D108216F
:104AC000BA688A43BA60BA689A43BA6008227C4CD2
:104AD0002388934323802188402089B2FCF750F833
:104AE0002A00238880329BB213806E4B6A4C1E7062
:104AF000002363700533A370704B1888714B80B22C
:104B00001988714B89B21A8892B2FCF78FF9E0705C
:104B100017E06C4B108819885F4C884202D1412302
:104B200063700BE00521217010881988664B80B2F4
:104B30001A8889B292B2FCF779F960700222594B57
:104B40001A70624B4C331B88052B01D0FDF7CCFF4C
:104B50002021514A53780B4353705D4A0B991368D7
:104B60000B4013605B4B5C4A1A600F2299680A4045
:104B700080219A60594A93688B439360FDF7B4FF94
:104B80002300574D7A3319882A88914226D08022F3
:104B90001B889BB22B804A4B1B889343484A40207A
:104BA00013801188803489B2FBF7EAFF444B1B88DD
:104BB0009BB223803B4B384C1E700023637005333F
:104BC000A370344B28881988464B80B289B21A8862
:104BD00092B2FCF72BF9E070FDF786FF2D4B298888
:104BE0001A882D4C914202D1412363700BE00522BB
:104BF0002270288819883B4B80B289B21A8892B2F9
:104C0000FCF714F960700222264B1A70FDF76CFF56
:104C10009C785D782D4AEDB2ABB205936B1C5B00BE
:104C2000985AABB2E4B280B2632B09D92B00633B34
:104C30005B00985A642180B206F0B2FE80B207E0B1
:104C4000ABB2273B182B03D8642106F02FFF88B2A4
:104C5000A3B20593174B1A780C231340082B06D0E8
:104C60000C2B5ED0042B01D0FDF75DFF4BE01F2322
:104C700022009A43E02A01D0FDF755FF07220023C6
:104C80000121224093422FDA49000133C9B2DBB23D
:104C9000F8E7C0467C040020C9050020600700201A
:104CA00090040020A104002068070020FFFFFFBF40
:104CB0001407002061040020804000506607002097
:104CC000E80100209E040020B404002020020020FF
:104CD000200A002000400050FF0F0000C04000509C
:104CE000FA060020160A0020E30601D5FDF71BFF97
:104CF000082308401C4001D000280AD10443E4B234
:104D0000002C08D105E00023BB60059BC0B28342A4
:104D100001D1FCF743F8FA22114B92001A60FDF71B
:104D200002FFABB20524062B11D005992800FBF732
:104D30005FFF059B83420AD0013CE4B2002CF4D112
:104D4000084B984203D1FBF70DFF00F0AFFDFCF7D5
:104D500025F8FBF707FF00F0A9FDFDF7E4FEC046CC
:104D6000BC040020FFFF000007B5094A136A009346
:104D7000084B196A019100991162019A1A62064B57
:104D80001B68002B02D000980199984707BDC046C8
:104D900000400050404000500C0100201FB50C2482
:104DA0000D480E49036A0E4A01930B6A0293136A77
:104DB0000393029BA3430293019B0362029B0B623A
:104DC000039B1362074B5B68002B03D00198029989
:104DD000039A98471FBDC04680400050C040005015
:104DE000004100500C0100200422044B10B51A624F
:104DF000034B9B68002B00D0984710BDC04000506B
:104E00000C0100200822044B10B51A62034BDB682A
:104E1000002B00D0984710BDC04000500C0100206E
:104E2000094B800182B0C01801900198019B1A685B
:104E300001238B402021134303600020034A1368A1
:104E40000B43136002B07047144000508041005083
:104E500010B50F2811D80F23094A184014689C4335
:104E60000E3B19400B01102120431060106888434D
:104E7000010019431160002000E0024810BDC04647
:104E8000804100500189FFFFF7B5274C01940029AC
:104E900007D1019D019906000C6801211036B1402F
:104EA00012E0012904D1019D019C814024680BE09E
:104EB00002290BD1019D019906000C6801210F0008
:104EC0001036B74081403943214329601749019189
:104ED000019C0121002A05D18140019A12688A4370
:104EE000226004E08140019A126811432160C021D0
:104EF0000F4C104A8900022809D15058A3600E4B6C
:104F000003408020000403435350042308E0802022
:104F1000E360535800061B021B0A03435350082347
:104F200000201360FEBDC046DC400050D840005059
:104F30000C01002000E100E0FFFF00FF30B5031E80
:104F40001D2B00D9C6E006F017FD0F1B22292B32BE
:104F5000323232323232323E444A50565D637180D0
:104F60008080808E8EA19ABC00205B4B18605B4BCA
:104F700018605B4B18605B4B18605B4B1860AAE0D5
:104F8000584A5A4B11680B408021C9019EE0554A8E
:104F9000574B11680B40C021890197E04F4A00E050
:104FA0004D4A1168534B0B40F02109028EE001225B
:104FB0001500DC1CA540053B9A4048480168A94300
:104FC0000A43026084E0474A4B4B11680B400421BE
:104FD0007CE0444A494B11680B40082176E0414A85
:104FE000474B11680B40102170E03E4A454B116859
:104FF0000B4020216AE0394A434B11680B40802165
:10500000490063E0354A414B11680B4080211AE0AA
:10501000344A3F4B11680B4003210B4313602E4A67
:105020003C4B11680B40C02109014FE02B4A394B22
:1050300011680B40C02109010B431360264A344B11
:1050400011680B40C021890040E0113B5900032347
:105050000C001D00083C8B40A5402148026813430A
:10506000AB43036034E0204A1168192803D1284B70
:105070000B4003212AE0274B0B400C2126E0FF21A7
:10508000174A13681B0C1B040B431360FF21124AC1
:1050900013681B0C1B040B431360124A174B116857
:1050A0000B40802109010B43136011681A4B0B4020
:1050B000C0210B4313600C4A0D4B11680B4030218B
:1050C00004E0094A144B11680B40C0210B431360E4
:1050D000002000E0114830BD300000503400005086
:1050E000380000503C00005040000050BFBFFFFFA0
:1050F000CFCFFFFF0F0FFFFFFBFBFFFFF7F7FFFF18
:10510000EFEFFFFFDFDFFFFFFEFEFFFFFDFDFFFF15
:10511000FCFCFFFFF3F3FFFF3F3FFFFF0189FFFFB1
:10512000F8B501232A4C25681D4205D02360294B80
:105130001B68002B00D0984702231D4205D0236036
:10514000244B9B68002B00D0984704231D4205D0B8
:105150002360204B1B69002B00D0984708231D4279
:1051600005D023601B4B9B69002B00D098471A4D3C
:105170001A4C2F682668FB0608D52A68184B13407E
:105180002B60144B5B68002B00D09847FB0208D5BE
:105190002A68144B13402B600E4BDB68002B00D0A9
:1051A0009847F30608D522680D4B13402360094B3E
:1051B0005B69002B00D09847F30208D52268094BA1
:1051C00013402360034BDB69002B00D09847F8BDE8
:1051D000440004401C0100205000044054000440DE
:1051E0001F000F000F001F00F8B501232A4C25688F
:1051F0001D4205D02360294B1B6A002B00D0984725
:1052000002231D4205D02360244B9B6A002B00D053
:10521000984704231D4205D02360204B1B6B002BB5
:1052200000D0984708231D4205D023601B4B9B6B81
:10523000002B00D098471A4D1A4C2F682668FB06A1
:1052400008D52A68184B13402B60144B5B6A002B5F
:1052500000D09847FB0208D52A68144B13402B60F6
:105260000E4BDB6A002B00D09847F30608D5226866
:105270000D4B13402360094B5B6B002B00D098470C
:10528000F30208D52268094B13402360034BDB6B04
:10529000002B00D09847F8BD440014401C010020AA
:1052A00050001440540014401F000F000F001F0056
:1052B000F021084A090413680B43C0211360064B10
:1052C00089031A680A431A601968044A0A401A6076
:1052D0007047C046080200500C000050FFFFCFFF8F
:1052E00007230340043BDAB230B5032A0ED9382431
:1052F000C5002540373CAC4000251E4A1368A34337
:10530000A94200D025002B4313600CE001251A4C64
:10531000DB0022689D4013000022AB43914200D085
:105320002A0013432360C30622D5103807281FD84C
:1053300006F022FB0406080A0C0E10160F4A0AE0BB
:105340000E4A0EE00E4A06E00D4A0AE00D4A02E05F
:105350000C4A06E00C4A11680C4B0B40082105E092
:10536000094A11680A4B0B40802109030B43136063
:1053700030BDC046080004400800144050000440FE
:1053800054000440500014405400144007000F0023
:105390000F00070007230200F0B51A4085B0019204
:1053A000023A00900D00AC4B052A05D8100006F01B
:1053B000E3FA060608080B0B5B699B0006E05B69D5
:1053C00004E0DB699B0601E0DB691B069B0F04D050
:1053D000022B04D1A14B1B6802E0A14B00E0A14BC2
:1053E0000293009B172B40D8180006F0C5FA0C0C4E
:1053F0000C0C121212123E3E3E3E3E3E3E3E222417
:1054000026282A2C2E36009B9748DC00016802349F
:1054100004E09648009B0168DC001E3C0123A34089
:105420000024EE689943A64200D01C0023000B43E1
:105430001AE08F490AE08E4810E08E4906E08D4858
:105440000CE08D4902E08C4808E08C4908688C4BE0
:105450000340E86803430B6007E08848E968036895
:105460000C0487490B4023430360019B2E781F1FC8
:10547000FBB2032B11D900997B48CC003821214085
:10548000012403318C4003682100A3430024A64279
:1054900000D00C00234303600CE00120FC00033427
:1054A000A040002471490B688343A64200D0040049
:1054B00023430B606968002966D1EB78052A05D87B
:1054C000100006F059FA050507070C0C6D4902E0BB
:1054D0006C4905E06C49FF200A68824304E06A4990
:1054E00008681A02694B034013430B606878AC6884
:1054F0006421604306F054FAAA78FBB201380392A3
:10550000032B18D9009A624B91001C221140153AC6
:1055100017008F401E68BE43039F17403A008A4021
:1055200016431E600C23019A611E5343594A9A1870
:105530001160594A14E0594BBA00196807231E003C
:105540009640B143039E1E40330093401943534B92
:10555000534A19600C237B43611E9A181160514A0B
:105560009B181860AB780126032B01D84E4AD65CF5
:10557000E9780298013106F013FA310006F010FACA
:10558000210006F00DFAF9E0029806F009FA8023EE
:1055900007005B0500209F4200D9EFE0434B9F428C
:1055A0002ED9390C38008CB206F0FAF980235B0250
:1055B000984201D90134A4B280235B009C4220D9D7
:1055C0003C0A390E2000CEB206F0EAF980235B02D5
:1055D000984201D90136F6B2002301200200591C7D
:1055E0009A40CBB2B242F9DD0126013B9E40F6B2B1
:1055F0000020102E00D9C1E027028024640001E0C1
:10560000022401262100380006F0CAF9310006F014
:10561000C7F9070083B221000298039306F0C0F98E
:10562000310006F0BDF9B9B206F0BAF9019B02905B
:10563000981E013C052804D806F09EF905050707C9
:105640003A3A104A02E00F4A33E00F4AFF2113684A
:105650000C408B4332E0C046000200501C0000208A
:10566000001BB700008051010800044008001440EE
:1056700050000440540004405000144054001440B2
:105680000F000F000000044000001440FF00FFFF67
:10569000040004400C0004401000044004001440C6
:1056A0000C001440100014409CBD0000FFFF0100DE
:1056B000334AE4B211682302324C0C401C43701E82
:1056C00014600F2812D806F057F91008110A1111AA
:1056D000110C111111111111110E002606E00126F5
:1056E00004E0022602E0032600E00426009B68781E
:1056F000DB0607D5AB6864215F1E5843BFB206F0D6
:105700004FF907E0039B013F434364211800BFB2F8
:1057100006F0D0F9019B01381A1FD3B280B2032BD7
:1057200017D9009B184C99001C231940153B1D00EC
:105730001E408D408E4022680533AA4332432260CA
:10574000019A5343114A9A181760114A9B1818601E
:1057500013E007219500A9400E4C23688B431900E4
:1057600007231E40AE4005335A430B4B3143D31839
:1057700021601F60094BD2181060029805B0F0BD7F
:1057800000001440FF00FFFF040004400C00044030
:1057900010000440040014400C0014401000144099
:1057A0001023042200291CD018420ED0104204D02D
:1057B0001C4914388A6F0F3B04E007231A4918402C
:1057C0008A6F063B834013431BE00123104203D042
:1057D000164904380A6801E015490A6883401343F2
:1057E0001DE018420FD0104204D00E4914388B6FC0
:1057F000033A04E007220C4910408B6F063A8240BE
:1058000093438B670CE00123104203D0074904380F
:105810000A6801E006490A6883409A4313000B6056
:105820007047C04600001440000004407C00144053
:105830007C00044007221040023800B50323124ABE
:10584000052804D806F098F80909111116160B401E
:10585000506919070D4B034004E050690B4099074C
:1058600083009B080B4353610CE00B401901D06986
:10587000302303E00B409901C023D0699843030013
:105880000B43D36100BDC04600020050FFFFFFCFB5
:105890000022044B5A60586801231840904200D0FF
:1058A00001487047FC0000500296FFFFA022012132
:1058B000D20593680B43936070470000A02210212B
:1058C00010B5D20593690B439361034B1B68002B02
:1058D00000D0984710BDC0465C01002010B50728D5
:1058E00019D8031F022B16D9012814D007210B4BFE
:1058F00008401A698A4310431861D8680006C40F2B
:1059000005D0DA6879310A43DA60054804E002F02C
:105910000FFA200000E0034810BDC046000200500E
:105920000796FFFF0396FFFF402110B5044A136856
:105930000B431360034B5B68002B00D0984710BDEE
:10594000000200505C01002000487047001BB700B7
:1059500030B585B06A46134B6D4613CB13C21B6836
:105960001360114B1A6A120301D4104A00E0104A66
:105970001B6A0D4C0020DB0311D4206A216A246AC3
:10598000C005C00D89042404C90EA40F02300231E1
:105990005043A40006F004F8295906F001F805B0B8
:1059A00030BDC046A0BD000000020050001BB70083
:1059B0000080510110B50E4C23695B070ED023699E
:1059C0005B075B0F022B02D1FFF7C2FF09E02369DF
:1059D0005B075B0F032B03D0064802E0064800E09C
:1059E0000648A1690907090F013105F0D9FF10BD6B
:1059F0000002005000805101001BB700102700007A
:105A00000022074B1B685843064B58609A600532CA
:105A10001A608022520219681142FCD07047C046B9
:105A20002000002010E000E00022F0B50125B94B75
:105A300019681A60B84A146813002C4000D080E23C
:105A40007D2900D845E11A21B448056912688A43C6
:105A50001A60B34AB3491470043425424CD0CD685F
:105A600006692642FCD1CC681678651BAE4CB600A0
:105A700035512E00293E2B2E00D840E2C82D00D9EA
:105A800027E215780135EDB21570A64DEE680425B4
:105A900007692F42FCD0CD68AD1B1678B600A55122
:105AA000C82D00D915E2042615780135EDB2157020
:105AB0001578212D1AD8CF6805693542FCD1CD68FB
:105AC000EF1B1578AD00675115780135EDB21570F3
:105AD000CF6805693542FCD0CD68EF1B1578AD0065
:105AE000675115780135EDB21570E1E70426CD68F0
:105AF00007693742FCD14BE0CD6806692642FCD0ED
:105B0000CE68894C761B1578AD002E51157801357D
:105B1000EDB215703500293D2B2D00D8EFE1C82ED0
:105B200000D9D6E17F4DEE68042507692F42FCD1EC
:105B3000CD68AD1B1678B600A551C82D00D9C8E1B7
:105B4000042615780135EDB215701578212D1AD877
:105B5000CF6805693542FCD0CD68EF1B1578AD00E4
:105B6000675115780135EDB21570CF68056935427A
:105B7000FCD1CD68EF1B1578AD0067511578013564
:105B8000EDB21570E1E70426CD6807693742FCD015
:105B9000002080260127C9681278491B9200A15075
:105BA000624A6349604D1060B60208608400A446F2
:105BB00038420AD014686408146064462C59502C8A
:105BC0000DD90C6834430C6009E00C6864080C6063
:105BD00064462C59502C02D91468344314600130A7
:105BE0002328E3D11C68534820401860106800281F
:105BF00003D10868002800D16BE1106809680142F0
:105C00005BD1C02110688900084256D180201968F4
:105C100000040143196011684748C9B2405C474914
:105C200008601168890A1160126845493F2A3AD014
:105C300011D80F2A2BD006D8032A24D00C2A2AD018
:105C4000002A36D134E0332A29D03C2A2DD0302AFC
:105C50002FD104222CE0CF2A1BD007D8C32A14D07E
:105C6000CC2A1AD0C02A24D1082221E0F32A18D045
:105C700003D8F02A1DD10C221AE0FC2A17D0FF2AE3
:105C800017D10F2214E0012212E0092210E00322B2
:105C90000EE00B220CE002220AE00A2208E00522B4
:105CA00006E00D2204E0072202E0062200E00E22B8
:105CB0004A704A782349D2B24A701968224A0A4087
:105CC0001A601A6821490A431A600422204BDA67D5
:105CD00037E1022900D834E11068800700D4F6E0EB
:105CE0001068C0063AD51B4A1078A84310700829DE
:105CF00003D811780131C9B21170174908781178A9
:105D0000414011701278D20700D5E2E010211A68E4
:105D10008A43ACE06401002068070020C0400050C6
:105D20001C0A00200000114070070020F00600202F
:105D300054070020FFFF7FFFB0BD0000FC010020E2
:105D4000EA0100206104002001FFFEEF01000800CD
:105D500004E100E064070020880400201068800649
:105D600000D497E00420146804420CD14024136846
:105D7000034313601068A0431060082900D9E0E0D5
:105D800013682343B1E080241068A0431060082901
:105D900002D8126822431A6040211A681868520813
:105DA0000A4001408A4200D0CBE004211A68654CC9
:105DB0008A431A6018686449644A000659D5107805
:105DC0002478C0B2E4B20C54002004001578A84234
:105DD00004D80D5C01306C40C0B2F7E7002C43D111
:105DE0004878002812D1087800280FD110780028B0
:105DF0000CD01968564A0A4048211A60554A9160E9
:105E0000554AB83114601A680A4310E01868C00592
:105E100005D50F240878A043702805D109E03F2458
:105E20000878A043802804D019684C4A0A401A60B8
:105E30004FE01868800005D51868C00502D41868BE
:105E4000474C01E01868474C204318600020464D3D
:105E50001478A04205D20C5CE4B22C540130C0B2DC
:105E6000F6E70421414AD1671968414A0A401A609D
:105E700067E010782478C0B2E4B20C54202019688E
:105E80008143196011780131C9B211701278102A5A
:105E90001FD856E02B4802785200D2B2027008296F
:105EA00003D802780132D2B2027032490A78013244
:105EB000D2B20A700A78072A05D920201A6802434C
:105EC0001A6000220A7010211A680A43CFE70329DA
:105ED0000DD11968284A0A401A600023254A137018
:105EE0001A4A1370254A1360254A136029E00929CC
:105EF00005D8204A13780133DBB2137021E01D4A24
:105F000011781229E5D91968490707D502201968BF
:105F10000143196018681B49014019600420196881
:105F200001431960196889070BD5196800180143E6
:105F30001960186814490140196000231370034A5E
:105F4000DBE7F0BD88040020EA010020C205002044
:105F5000FFDFFFFFC040005080400050FFF6FFFF12
:105F600001000810010008006104002004E100E0C5
:105F70000FFFFEFF1C0A002000FFFEFFF0060020BE
:105F800054070020FFFFFEFFCBFFFEFFF0B52F4BB5
:105F90002F4A1B781168002B13D180202D4B8003D2
:105FA0000B401360136880214340136012682A4B32
:105FB000024202D19A688A4301E09A680A439A60D1
:105FC00042E080240525254BA4020B401360136892
:105FD000234F63401360234B1878C0B2411CC9B2F1
:105FE000197021490D541878C0B2451CEDB21D70CE
:105FF00004250D541878C0B2451CEDB21D70002563
:106000000D541878C0B2451CEDB21D703D78EDB24C
:106010006E1CF6B23E700D541878C0B2451CEDB23D
:106020001D7087250D541878C0B2451CEDB21D7047
:1060300013689B03DB0F0B541368234204D18021A8
:10604000054A93688B439360F0BDC0463D0A00202B
:1060500068070020FFFFFDFFC0400050FFFFDFFF8B
:10606000E806002016020020CF05002070B50125AB
:10607000B94ABA49936808002B4393600B68B84A41
:106080005B190B60136814001B0300D463E10B79E8
:106090005B19DBB20B710A2B00D1B3E00AD8032BDA
:1060A0003FD002D8AB4224D055E1062B51D0082B6B
:1060B00063D050E1142B00D1E7E006D80C2B00D1BF
:1060C000B2E00F2B00D1CAE045E1192B00D125E148
:1060D0002A2B00D03FE11068A24B0340042013603C
:1060E000A14BA24A186093688343936000230B710D
:1060F00031E19F4B1B68002B00D12CE180211368FC
:10610000C9000B4313603F229A489B4903889B09AF
:106110001340CC5C994B1C70008802408A5C5A701A
:1061200019E11368DB0500D415E104218E4B1960D9
:10613000002393498B6093490B60106889490140A3
:1061400011604821904A9360904A9160904A936010
:1061500001E19048037840781B021B188B608E4940
:106160008B4200D0F7E0824B1B68002B00D0F2E09E
:1061700011688A4B0B401360EDE01368DB0000D41C
:10618000E9E00421794A93680B439360784B1A68DD
:10619000002A00D1DFE01968814A114212D0FF22A3
:1061A00019689201114205D00722196802737D4ACD
:1061B0000A401A600F211A680A4200D1CBE0062279
:1061C000027309E010211A680A4209D0764A017365
:1061D0005278120700D5BEE01A688A431A60BAE006
:1061E00020211A680A4200D1B5E06F4A0173527843
:1061F000120700D5AFE01A688A431A6023685B0073
:106200005B08A7E013685B0500D4A4E01368DB001B
:1062100000D4A0E0654B1B8F2B4200D19BE00221F4
:106220005648FAF785FD96E0614B1B78032B00D8A2
:1062300091E00F21574B9A788A43E02A00D08AE0F8
:106240005C4A10781978884200D084E052785B78F4
:106250009A4200D07FE080222368920079E01368A0
:106260009B0578D51168544B0B4013600222534BA9
:106270004E491A700023524A1370464BDB780133A3
:106280005B005B5ADBB2537065E013685B0513D5A6
:1062900012684C4B8E68404D134023600620474ADD
:1062A000474B097BAE4203D118705970022302E0BC
:1062B0009870D970042313702368DB004BD53F4BD3
:1062C0001B78012B47D93F243D492C4B0A7892007B
:1062D000D2B21A704A78187892098218D2B21A701B
:1062E0004A78254822405A701A78825C1A705A7887
:1062F000825C5A708A789200D2B29A70CA789D787D
:106300009209AA18D2B29A70CA781440DC709A78AE
:10631000825C9A70DA78825CDA701CE0234B1B8F07
:106320009B0703D412681D4B134023602368DB00D6
:1063300011D5224B1A78002A0DD019780F48C9B20E
:10634000FAF7F6FC2268154B13408022236023687D
:10635000D2051343236070BD00000140640100209A
:1063600068070020FFFFF7FF00E100E00040005059
:10637000200A002086040020B0BE0000C3050020D3
:10638000004100503800005040400050C0400050D4
:1063900080400050610400200FBF0000FFFFFFEFAE
:1063A000CF7F00003FC0FFFFEA0100202002002055
:1063B000C20500205F040020FFFDFFFFA1040020B4
:1063C000C9050020FFFBFFFFF7B58C4D8C4A2B88D9
:1063D00001339BB22B801388002B03D01388013B21
:1063E0009BB21380874A1388002B03D01388013B8C
:1063F0009BB21380844A1378002B03D01378013B9F
:10640000DBB21370814C2368002B0FD02368012B63
:1064100009D148227E4B9A6000227E4B9A60FAF79F
:10642000A1FBFFF743FA2368013B23607A4B1A78FC
:106430000093002A1FD0794B1A6801321A601A683B
:10644000FA239B009A4216D9754B04211A680F2330
:106450001340744A403313700023009A1370724A39
:106460001370724A1370724B9A680A439A609A6862
:1064700002390A439A606F4A1378002B03D01378CD
:10648000013BDBB213706C4F3B689B0400D484E08B
:106490003B68DB0500D580E0684C23004C331A884C
:1064A00092B2042A1FD120205A4B996881439960E7
:1064B0009968103881439960996870308143996078
:1064C000996840388143996099683E388143996062
:1064D00099680138814399609968073081439960D0
:1064E00099689143996096232A885B009A4204D95F
:1064F0004021474A93688B439360FA232A88DB0044
:106500009A424AD93A684E4B13403B60230082338B
:106510001B88DB0703D54B490020FAF753FC230007
:1065200082331B889B0703D546490120FAF74AFCB2
:10653000230082331B88DB0603D542490420FAF787
:1065400041FC230082331B889B0603D53D4905206F
:10655000FAF738FC230082331B885B0703D53949DF
:106560000220FAF72FFC230082331B881B0703D578
:1065700034490320FAF726FC230082331B885B068C
:1065800003D530490620FAF71DFC823423881B0608
:1065900003D52C490720FAF715FC00242A4A660087
:1065A00013000E33F35A0192002B0AD0012B03D1B2
:1065B000E0B22449FAF706FC019B0E33F25A013A85
:1065C000F2520134082CE9D13B689B020AD52B8892
:1065D0000F4980229B0502D58B68134301E08B682D
:1065E00093438B603B689B0333D52B8808498022FB
:1065F000DB052BD58B6813432AE0C0465A070020E1
:10660000840400205C07002075040020BC040020E6
:10661000C0400050004100503D0A0020380A0020D0
:10662000E4010020C105002016020020320A0020EB
:1066300000001540A0040020680700202002002070
:10664000FFDFFFFFFFFF0000640100208B68934322
:106650008B60B34E3368DB0628D52B881B0504D12D
:106660008021B04A93680B4393602B881B051B0D58
:10667000802B03D1AB498A689A438A6080222B8899
:1066800052001B051B0D934204D18021A54A93683B
:106690000B439360C0222B8852001B051B0D9342B5
:1066A00004D180219F4A93688B43936033689B0693
:1066B00058D52B881B0504D180219A4A93680B4337
:1066C00093602B881B051B0D802B03D195498A688D
:1066D0009A438A6080222B8852001B051B0D93422F
:1066E00004D180218F4A93680B439360C0222B888A
:1066F00052001B051B0D934204D18021894A9368E7
:106700008B43936080222B8892001B051B0D9342C4
:1067100004D18021834A93680B439360A0222B8885
:1067200092001B051B0D934204D180217D4A936882
:106730008B439360C0222B8892001B051B0D934254
:1067400004D18021774A93680B439360E0222B8821
:1067500092001B051B0D934204D18021714A93685E
:106760008B439360704C23004C331B88002B00D06C
:106770008FE00122336813421DD0230084331B882D
:10678000134218D0E388002B15D02389002B12D098
:1067900080212B8889009B059B0D8B4203D1634987
:1067A0008B6893438B602B889B0504D101215F4A42
:1067B00093680B4393600222336813421DD0230079
:1067C00084331B88134218D06389002B15D0A3890A
:1067D000002B12D080212B8889009B059B0D8B42BA
:1067E00003D152498B6893438B602B889B0504D15E
:1067F00002214E4A93680B439360042332681A4285
:1068000020D0210084310988E21819421AD0D38F90
:10681000002B17D0A31DDB8F002B13D080222B88D9
:1068200092009B059B0D934204D110213F4A93682F
:106830008B4393602B889B0504D110213B4A9368BE
:106840000B439360082332681A4222D0220084321C
:1068500012881A421DD023000833DB8F002B18D07A
:10686000230048331B88002B13D080222B889200F2
:106870009B059B0D934204D120212C4A93688B43A6
:1068800093602B889B0504D12021284A93680B43F1
:106890009360274A1388002B03D01388013B9BB2D7
:1068A0001380244B1988002903D01988013989B233
:1068B000198021480188002903D00188013989B253
:1068C00001801E480188002903D00188013989B25E
:1068D00001801B480188002903D00188013989B251
:1068E000018018480188002903D00188013989B244
:1068F000018015480188002903D00188013989B237
:10690000018012480188002903D00188013989B229
:1069100001803968002923DA0D4801781AE0C04661
:10692000200A0020C040005020020020804000507B
:106930009A040020820400208A040020E606002039
:10694000EC060020120800205E070020140700203B
:1069500076040020002903D001780139C9B2017002
:10696000E188002917D01288002A14D10121A44AF5
:10697000107808420FD02027A24DA868B843A8601D
:10698000107888431070009A1278032A03D19E4829
:1069900002880A4302802289002A17D01B88002B14
:1069A00014D10222964B197811420FD01025954828
:1069B0008168A9438160197891431970009B1B7805
:1069C000032B03D190490B8813430B806389002B61
:1069D00018D08E4B1B88002B14D10422884B1978B9
:1069E00011420FD0802587488168A94381601978BA
:1069F00091431970009B1B78032B03D182490B88AC
:106A000013430B80A389002B18D0814B1B88002BCC
:106A100014D108227A4B197811420FD040257948B9
:106A20008168A9438160197891431970009B1B7894
:106A3000032B03D174490B8813430B80231DDB8F79
:106A4000002B18D0734B1B88002B14D110226C4BD9
:106A5000197811420FD002256A488168A9438160E4
:106A6000197891431970009B1B78032B03D1664959
:106A70000B8813430B80A31DDB8F002B18D0664BB4
:106A80001B88002B14D120225D4B197811420FD0A6
:106A900001255C488168A943816019789143197088
:106AA000009B1B78032B03D157490B8813430B80A2
:106AB00023000833DB8F002B18D0584B1B88002B8A
:106AC00014D140224E4B197811420FD008254D4861
:106AD0008168A9438160197891431970009B1B78E4
:106AE000032B03D148490B8813430B802300483301
:106AF0001B88002B1AD04A4B1B88002B16D1404B09
:106B00001A7852B2002A11DA04203E498A68824378
:106B10008A607F2219780A401A70009B1B78032B29
:106B200004D18021384A13880B4313803D4D3E4FDA
:106B30002A883B889A4256D23C4A1378002B02D0CE
:106B4000013B13704FE00A231370394B1A882B88CE
:106B5000D3189BB22B802A883B889A4202D93B8863
:106B60009BB22B802988002089B2FAF72BF92A885A
:106B70003B889A4237D12F4B1B78032B05D18021BC
:106B8000214A490013880B4313802B4A13685B008A
:106B90005B08136023004C331B88042B04D1202195
:106BA000184A93680B439360230082331B88DB07EA
:106BB00006D5230086331A88642353431F4AD381A2
:106BC00023004C331B88052B0DD180211C4B1B69E6
:106BD0000B4208D1802332685B001A433260194AA5
:106BE00093680B4393602A883B889A4200D87BE0E5
:106BF0000E4A1378002B27D0013B137074E0C04677
:106C000060070020004100508C0400208A0400200E
:106C1000E6060020EC060020120800205E07002097
:106C20001407002078040020E40600200000002063
:106C3000340A00203D0A002068070020640100207B
:106C400040400050C04000500A231370B94B1A88CE
:106C50002B889B1A9BB22B802A883B889A4202D2AF
:106C60003B889BB22B802988002089B2FAF7AAF8CA
:106C70002A883B889A4237D1AF4B1B78032B05D12A
:106C80008021AE4A490013880B431380AC4A136835
:106C90005B005B08136023004C331B88042B04D17A
:106CA0001021A84A93680B439360230082331B880A
:106CB000DB0706D5230086331A8864235343A24A90
:106CC000D38123004C331B88052B0DD19F4B1B69AF
:106CD0005B0609D4802280213368520013439C4A0A
:106CE000336093680B4393609A4D9B4E2A88338898
:106CF0009A4258D2994A5378002B02D0013B5370E4
:106D000051E00A235370964B1A882B88D3189BB2F4
:106D10002B802A8833889A4202D933889BB22B80F1
:106D20002988012089B2FAF74DF82A8833889A42D7
:106D300039D1814B1B78032B05D180217F4A8900F3
:106D400013880B4313807E4A13685B005B08136053
:106D500023004C331B88042B04D18021794A93688B
:106D60000B439360230082331B889B0706D52300C7
:106D700086331A8864235343734A138223004C33A7
:106D80001B88052B0FD1714B1B699B060BD48021EF
:106D9000744A890013680B4313606D4A8139936804
:106DA000FF390B4393602A8833889A4258D96B4A3B
:106DB0005378002B02D0013B537051E00A235370EB
:106DC000674B1A882B889B1A9BB22B802A883388A2
:106DD0009A4202D233889BB22B802988012089B243
:106DE000F9F7F0FF2A8833889A4239D1524B1B7841
:106DF000032B05D18021514A890013880B4313804E
:106E00004F4A13685B005B08136023004C331B88F8
:106E1000042B04D140214B4A93680B439360230019
:106E200082331B889B0706D5230086331A88642388
:106E30005343454A138223004C331B88052B0FD143
:106E4000424B1B69DB060BD48021464A890013683C
:106E50000B4313603E4A81399368FF390B439360BB
:106E6000414D424E2A8833889A4257D23B4A937802
:106E7000002B02D0013B937050E00A2393703C4BEF
:106E80001A882B88D3189BB22B802A8833889A4281
:106E900002D933889BB22B802988022089B2F9F766
:106EA00091FF2A8833889A4238D1234B1B78032BD1
:106EB00005D18021214AC90013880B431380204A41
:106EC00013685B005B08136023004C331B88042BA2
:106ED00004D102211B4A93680B4393602300823341
:106EE0001B885B0706D5230086331A886423534327
:106EF000154A538223004C331B88052B0ED11D4BA2
:106F00001B699B060AD48021164AC90013680B43EB
:106F1000802113600E4A93680B4393602A8833885C
:106F20009A4200D879E00D4A9378002B24D0013B97
:106F3000937072E0340A00203D0A00208C04002087
:106F400068070020004100506401002040400050CC
:106F5000C0400050F60600207A0400200000002007
:106F600062070020200A0020180A00209804002050
:106F7000B6040020004000500A239370A94B1A88E1
:106F80002B889B1A9BB22B802A8833889A4202D284
:106F900033889BB22B802988022089B2F9F712FF2F
:106FA0002A8833889A4238D19F4B1B78032B05D10E
:106FB00080219E4AC90013880B4313809C4A1368A2
:106FC0005B005B08136023004C331B88042B04D147
:106FD0000121984A93680B439360230082331B88F6
:106FE0005B0706D5230086331A8864235343924AED
:106FF000538223004C331B88052B0ED18F4B1B690A
:10700000DB060AD480218E4AC90013680B43802115
:1070100013608C4A93680B4393608B4D8B4E2A8888
:1070200033889A4257D28A4AD378002B02D0013B48
:10703000D37050E00A23D370864B1A882B88D3185C
:107040009BB22B802A8833889A4202D933889BB21C
:107050002B802988032089B2F9F7B4FE2A88338867
:107060009A4238D1704B1B78032B05D180216F4A8F
:10707000090113880B4313806D4A13685B005B089A
:10708000136023004C331B88042B04D10821694A68
:1070900093680B439360230082331B881B0706D53C
:1070A000230086331A8864235343634A93826A4BCE
:1070B0004C331B88052B0ED18020604B1B6903428B
:1070C00009D180235E491B010A681A430A605D4AA0
:1070D0009368034393602A8833889A4256D95C4A5E
:1070E000D378002B02D0013BD3704FE00A23D3703A
:1070F000584B1A882B889B1A9BB22B802A8833887E
:107100009A4202D233889BB22B802988032089B20D
:10711000F9F758FE2A8833889A4237D1424B1B78B8
:10712000032B05D18021414A090113880B431380A9
:107130003F4A4C3413685B005B08136023889BB2A2
:10714000042B03D13B498A6813438B60424B1A00DE
:1071500082321288120706D51A00863211886422FC
:107160004A4335498A824C331B88052B0ED1334B59
:107170001B695B060AD48021314A090113680B435D
:10718000802113602F4A93680B439360334C344D36
:1071900022882B889A423AD22D4A1379002B02D0AA
:1071A000013B137133E00A2313712E4B1A88238895
:1071B000D3189BB2238022882B889A4202D92B882D
:1071C0009BB223802188042089B2F9F7FBFD228835
:1071D0002B889A421BD1144B1B78032B05D180219D
:1071E000124A490113880B4313808021104AC903B6
:1071F00013680B431360184B1A0082321288D206B0
:1072000005D586331A88642353430B4AD3822288D8
:107210002B889A425BD90E4A1379002B24D0013B6C
:10722000137154E0B60400203D0A00208C040020B5
:107230006807002000410050640100200040005019
:10724000200A0020C04000509E0400206607002055
:1072500000000020B40400202002002010020020C2
:1072600000020020100800200A2313719C4B1A888A
:1072700023889B1A9BB2238022882B889A4202D2B1
:107280002B889BB223802188042089B2F9F79AFDCC
:1072900022882B889A421AD1924B1B78032B05D156
:1072A0008021914A490113880B4313808F4A136848
:1072B0005B005B0813608E4B1A0082321288D20684
:1072C00005D586331A88642353438A4AD3828A4C6D
:1072D0008A4D22882B889A4239D2894A5379002BC9
:1072E00002D0013B537132E00A235371854B1A8857
:1072F0002388D3189BB2238022882B889A4202D9F4
:107300002B889BB223802188052089B2F9F75AFD8A
:1073100022882B889A421AD1724B1B78032B05D1F5
:107320008021714A890113880B4313806F4A1368C7
:107330005B005B0813606E4B1A0082321288920663
:1073400005D586331A88642353436A4A13832288F7
:107350002B889A4239D96A4A5379002B02D0013BD3
:10736000537132E00A235371664B1A8823889B1AA3
:107370009BB2238022882B889A4202D22B889BB210
:1073800023802188052089B2F9F71CFD22882B88EB
:107390009A421AD1534B1B78032B05D18021524AB4
:1073A000890113880B431380504A13685B005B0804
:1073B00013604F4B1A0082321288920605D586332D
:1073C0001A88642353434B4A13834F4C4F4D2288F2
:1073D0002B889A4239D24A4A9379002B02D0013B3A
:1073E000937132E00A239371494B1A882388D3188A
:1073F0009BB2238022882B889A4202D92B889BB289
:1074000023802188062089B2F9F7DCFC22882B88AA
:107410009A421AD1334B1B78032B05D18021324A73
:10742000C90113880B431380304A13685B005B0863
:1074300013602F4B1A0082321288520605D586330C
:107440001A88642353432B4A538322882B889A42F9
:1074500039D92B4A9379002B02D0013B937132E04A
:107460000A2393712A4B1A8823889B1A9BB2238084
:1074700022882B889A4202D22B889BB223802188B3
:10748000062089B2F9F79EFC22882B889A421AD1ED
:10749000144B1B78032B05D18021134AC901138893
:1074A0000B431380114A13685B005B081360104B99
:1074B0001A0082321288520605D586331A88642350
:1074C00053430C4A5383134C134D22882B889A4202
:1074D00057D20B4AD379002B20D0013BD37150E017
:1074E000100800203D0A00208C04002068070020BE
:1074F0002002002064010020020200205807002022
:10750000000000207E040020F406002080040020FB
:10751000300A00207C040020FA0600200A23D371E0
:10752000374B1A882388D3189BB2238022882B8854
:107530009A4202D92B889BB223802188072089B2E6
:10754000F9F740FC22882B889A421AD12D4B1B78E0
:10755000032B05D180232C4A1B0211880B43138077
:107560002A4A13685B005B081360294B1A008232B9
:107570001288120605D586331A8864235343254A98
:10758000938322882B889A4239D9234AD379002BB6
:1075900002D0013BD37132E00A23D371184B1A8811
:1075A00023889B1A9BB2238022882B889A4202D27E
:1075B0002B889BB223802188072089B2F9F702FC2F
:1075C00022882B889A421AD10E4B1B78032B05D1A7
:1075D00080230D4A1B0211880B4313800B4A13684A
:1075E0005B005B0813600A4B1A0082321288120695
:1075F00005D586331A8864235343064A9383F7BD1F
:10760000160A00203D0A00208C0400206807002094
:1076100020020020640100200000002000228020C1
:10762000064B07499A608B6803438B6005497038A5
:107630000B6803430B60044B1A7070470041005005
:10764000C0400050200A002060070020384B10B5D1
:107650001A68002A07DB80211A6809060A431A60A3
:10766000C822344B1A80344C2378002B5ED1314A27
:10767000108880B2002804D01388013B9BB213808D
:1076800052E02E4B2E499860F9F79CFB2D4B2E4A69
:107690001B882B499BB201201380F9F793FB2B4BDE
:1076A0002B4A1B8826499BB202201380F9F78AFBDC
:1076B000284B294A1B8822499BB203201380F9F7E3
:1076C00081FB264B264A1B881D499BB20420138050
:1076D000F9F778FB234B244A1B8819499BB20520F4
:1076E0001380F9F76FFB214B214A1B8814499BB289
:1076F00006201380F9F766FB1E4B1F4A1B881049B2
:107700009BB207201380F9F75DFB80211B4B1C4ABD
:107710001B889BB213801B4A93680B4393601A4AE1
:10772000603913680B4313601423237010BDC046E7
:1077300068070020B8040020760400208040005034
:10774000FFFF0000E4060020780400207A040020F7
:10775000F606002098040020180A00206607002082
:107760009E04002000020020100200205807002084
:107770000202002080040020F4060020FA06002007
:107780007C040020C0400050200A0020024A1388D8
:1077900001339BB2138070471A0A0020F0B5B74836
:1077A00087B0036804AADBB2D11D0B7083690400A3
:1077B0001B07DD0F002B00DB45E108228369134323
:1077C00083614023087818403F33002800D1A6E0A9
:1077D00009780B407D2B00D19EE07E2B00D06CE21F
:1077E000A74D2B78002B77D1A6490B78DBB2002B65
:1077F00004D00B78013BDBB20B707DE20B21042639
:10780000A14DA248297001396970E631AB70EB7067
:107810002971B2396E71AB71E9710168090E297273
:107820000168090CC9B269720168090AC9B2A97272
:1078300001680C20C9B2E9729549087095490B702E
:1078400095498B77954B9649DE670868954B0340C1
:107850000B601021E3680B43E360E36849180B43B6
:10786000E360E3681A43E260A369DB00FCD52E788D
:10787000824BF6B21E60300000F0C2FA0127C0B29F
:10788000B74215D8A3691B02FCD4824A7B491378FE
:1078900001370133DBB21370EB5CFFB2DBB20B607C
:1078A0001378DBB2EB5C584000F0AAFAC0B2E7E70D
:1078B000A3691B02DB0FFBD1704A764910600A787E
:1078C0000132D2B20A70784A6D491370774A136058
:1078D00002220A70764A42E02B78022B00D00BE29B
:1078E00000F06CFA0021674A704B107071482970E3
:1078F000196019684C1C1C608142FAD9002119607A
:1079000013788B4200D0F7E1604B1B68DBB2137039
:107910000F2311780B4064E00022644B8CE00E785A
:107920001E421ED1644B1878C0B2002800D0E3E19B
:1079300080245D4964000B78DBB25A1CD2B20A7015
:107940005E4A5B009C520B785B0098520B7880215A
:10795000514ADBB293775A4A090613680B43136006
:10796000CAE1474B1B78DBB2022B67D0032B00D058
:10797000A3E1544B0D7819781F232B408B4200D084
:10798000BAE14A4B4C49186009780293002900D0AB
:10799000B2E1434B1B685B0100D5ADE1E3681031F8
:1079A0000B43E360E36810310B43E360E3681A4381
:1079B000E260A3693149DB00FBD5364A34481578CB
:1079C000037816009D4202D100230B6094E11378E6
:1079D0002D4DDBB2ED5CEDB22B1F3B2B03D90378B1
:1079E000DBB2137088E10D60280000F009FA01276E
:1079F000C2B2A3691B02FCD4337823490133DBB242
:107A00003370CB5C1D48DBB2036033780137DBB2E7
:107A1000C85CFFB2504000F0F3F9C2B2BD42E8D2F8
:107A2000A3691B02DA0FFBD1144BC0B21860337884
:107A30000133DBB23370029B1A605DE1164B9D7718
:107A40001A4B186039E11E4A1C4B1068002800DBF5
:107A50001BE1114FB87F40001E5AC020304033D088
:107A60001168490049081160BA7F0F49013AD2B242
:107A70000A700A780021520099523DE10000154039
:107A80003D0A0020C1050020CF050020E4010020B0
:107A9000160200203C0A00206401002004E100E0FE
:107AA00068070020FFFFFFFB320A0020380A002091
:107AB000200A0020FFFF0F006C07002014080020A0
:107AC000280A0020C00500208C4D2E78F5B20295C2
:107AD00002AE0135F571F579884E3570029D097851
:107AE0006E009953B97F4900595A002900D1E4E04A
:107AF000B97F824D49005E5AB97F2F7802318919CA
:107B0000C9B2B94200D0D8E02978C9B24E1CF6B249
:107B10002E7080264900B6005E5206002978490082
:107B2000585213685B005B081360754F754ABB7F42
:107B300039005B009B5A0133B3420FDBBB7FF31864
:107B4000DBB25B009B5A704ADBB29355935D013602
:107B5000584000F055F9F6B2C0B2E6E76B4A137828
:107B60001600DBB2022B06D0032B00D0A5E00022CA
:107B7000674B1A60A1E0644B002805D00023137006
:107B8000FF22644B1A70B7E01A791F00702A36D1B1
:107B900000225F4F60483A60597A0268120E9142A3
:107BA00000D08AE09A7AFF2194460268120C0A40BB
:107BB000944500D081E0DA7A94460268120A0A40BD
:107BC00094457AD11A7B00680840824275D103221D
:107BD00032705B79514ADBB213701378DBB2002B41
:107BE00001D133702AE000233B60444B4C4A1B78A0
:107BF000DBB213704B4A4C4B11680B405CE01A79B6
:107C0000722A1ED10025424A43481560597A0268FB
:107C1000120E914251D1FF219F7A0268120C0A4044
:107C200097424AD1DF7A0268120A0A40974244D149
:107C30001A7B03680B409A423FD13570354B19705F
:107C40005AE01878C2B201921A7894465A780132F2
:107C5000944532DD5A780132D2B28A778A7F9446CF
:107C600065461A78521BD2B21A700022013201986E
:107C7000D5B2854288D28D7F02A8AC469444654631
:107C80007D5D05700578BD54F0E71C48007801382B
:107C900040001E5A8020400086420ED11748174DE2
:107CA0000078C0B2461CF6B22E7009784000195216
:107CB0008021136809060B431360A3691B4A1B0448
:107CC00003D5022193680B439360A269174BD20737
:107CD00007D501219A690A439A619A6849180A43AB
:107CE0009A60A3699B0603D4104B9B69DB0603D5FE
:107CF0000222A3681343A36007B0F0BD320A00203C
:107D00006401002014080020C00400203D0A002067
:107D1000380A0020C1050020E4010020C005002031
:107D20003E0A002068070020FFFFFBFF000015400F
:107D300070B51B4C1B4D23695B075B0F052B02D8ED
:107D4000022B04D000E004239B00E85819E0012333
:107D5000266A3604B60FB3429B415B42F61A236A89
:107D60001B0301D4104B00E0104B206A216AC005B0
:107D7000C00D8904C90E02305843023103F010FED1
:107D8000F040A1690907090F013103F009FE084B12
:107D900068610849C01803F003FEA86170BDC046C1
:107DA0000002005008000020001BB70000805101B5
:107DB00020A1070040420F00704700000E4B1A78C8
:107DC00019785200D2B24A4052001978D2B24A40D1
:107DD00012011978D2B24A401978D20949005218D2
:107DE000D2B21A7018780F23044A18401378C018BA
:107DF0001F23184010707047EA060020E0010020A1
:107E00000023C20700D55E33820701D5BC22534050
:107E1000420701D561225340020701D5C2225340D7
:107E2000C20601D59D225340820601D5232253402C
:107E3000420601D54622534040B2002801DA8C2286
:107E400053401800704700008022BD49F0B50B6810
:107E5000D20413430B60BB4DBB4B97B01A782B7801
:107E60000C009A4200D093E18020B84AC0021588E5
:107E70001300002D00D1B6E00968014200D1B2E044
:107E800006A9497806A8017003201188014205D08F
:107E9000002306A98B711388834308E00C21148802
:107EA0000C4206D0012306A8837113888B431380EC
:107EB00092E0302114880C4201D00223F3E7C02461
:107EC0001188214004D006AB98711388A343EEE7D4
:107ED0001288D2050DD59E4A4C321288022A02D948
:107EE00006AA917102E0042206A98A711988994AAA
:107EF0005EE01A8892050CD5954A4C321288022A07
:107F000001D9012200E0052206A98A711988924A46
:107F10004EE01A8852050CD58D4A4C321288022A3E
:107F200001D9022200E0062206A98A7119888B4A2B
:107F30003EE01A8812050CD5854A4C321288022A76
:107F400001D9032200E0072206A98A711988844A10
:107F50002EE01A88D2040CD57D4A4C321288022AAF
:107F600001D9042200E0082206A98A7119887D4AF5
:107F70001EE01A8892040CD5754A4C321288022AE7
:107F800001D9052200E0092206A98A711988764ADA
:107F90000EE01A8852040DD56D4A4C321288022A1E
:107FA00001D9062200E00A2206A98A7119886F4ABF
:107FB0000A4010E01A8812B2002A0DDA644A4C32E4
:107FC0001288022A01D9072200E00B2206A98A7131
:107FD0001A885204520C1A80392306AA5371644B32
:107FE0001B789370A4E1236803425BD01022614E9A
:107FF0003368134256D033689B0653D509255E4B30
:108000001878C0B2421CD2B21A705C4A1554187863
:10801000C0B2451CEDB21D70082515541878C0B2C9
:10802000451CEDB21D70002515541878C0B2451CD2
:10803000EDB21D70524DAC4661462D78EDB26F1C0D
:10804000FFB20F70155418781021C0B2451CEDB264
:108050001D70BA2515541D78EDB2681CC0B2187099
:108060003068084046427041002180005055187821
:10807000C0B2451CEDB21D7011541878C0B2451C39
:10808000EDB21D70022515541878C0B2461CF6B228
:108090001E70802616541878C0B2461CF6B21E70A8
:1080A000155447E023685B0344D50120354B1A681B
:1080B00002423FD01A68344D82431A602B78002B5D
:1080C00038D006262C4B2E491878C0B2421CD2B2AA
:1080D0001A702A4A16541878C0B2461CF6B21E709E
:1080E000052616541878C0B2461CF6B21E7000263B
:1080F00016541878C0B2461CF6B21E700E78F6B24E
:10810000771CFFB20F7016541878C0B2461CF6B236
:108110001E70862616541878C0B2461CF6B21E7021
:10812000042616541878C0B2461CF6B21E702B787E
:10813000DBB21354236815491940216003F04FF94D
:10814000680700203E0A0020320A00208C0400202C
:1081500020020020FFFEFFFFFFFDFFFFFFFBFFFFF0
:10816000FFF7FFFFFFEFFFFFFFDFFFFFFFBFFFFF97
:10817000C0050020200A002016020020CF050020A4
:10818000E8060020280A00202E0A0020FFFFFFFB3F
:1081900080222B785200CE4E002B12D1FF33FF33BA
:1081A000F35A1100934202D18022520015E02B783D
:1081B000DBB25A1CD2B22A705B00F35A8B42F6D162
:1081C000F2E72B78013B5B00F35A9342ECD02B781B
:1081D000DBB2591CC9B22970F5E72B785B00F35A62
:1081E000934204D12B780133DBB22B70F5E72B7867
:1081F0005B00F35A002B75D02B785B00F35A0233E7
:10820000DBB20093009A2B78D318DBB25B00F25AF2
:1082100080239B009A4265D1002738002B78009A72
:10822000D318DBB25B00F752009AFBB29A420FD927
:108230002A78D2B2531CDBB22B705200B25AD3B29E
:1082400006AABB544340D8B2FFF7DAFD0137EBE78B
:108250002B780133DBB22B70002849D09D4B06AA46
:108260001B7892789A4243D1002106259A4B9B4F66
:1082700019701878C0B2421CD2B21A70984A1554BC
:108280001878C0B2451CEDB21D700525155418783C
:10829000C0B2451CEDB21D7011541D78EDB2681CC2
:1082A000C0B218703878C0B2461CF6B23E70505555
:1082B0001878C0B2451CEDB21D708625155418788B
:1082C000C0B2451CEDB21D70022515541878C0B21D
:1082D000451CEDB21D7006AB1B791354814B197010
:1082E000814B19602268814B1340236003F077F8BB
:1082F000784B06AA1B7892789A4219D17C4B1A784F
:10830000FF2A01D100221A701A7806A909790132D0
:108310008A420CD006AA5279012A08D00124754855
:108320000268224302601A787348D2B20270197050
:10833000684D06AC2B78A2789A4201D002F0D3FFA8
:1083400080226E4ED2043368310013433360627969
:10835000122A01D100F0B3FC00D959E1082A00D15A
:10836000BDE300D9CEE0042A00D13BE247D8022A7F
:1083700000D1F8E100D92EE2012A01D002F0B3FFCA
:108380000620554B1978C9B24A1CD2B21A70544A09
:1083900050541978C9B2481CC0B218700520505406
:1083A0001878C0B2411CC9B2197000211154187854
:1083B000C0B2441CE4B21C7011541878C0B2441C02
:1083C000E4B21C70812414541878C0B2441CE4B286
:1083D0001C70FE2414541878C0B2441CE4B21C7003
:1083E000AF23135401203D4B424A1870424B197081
:1083F0003F4B197013688343136002F074FF364BD0
:10840000062A00D12DE300D9F2E10B201978334E72
:10841000C9B24A1CD2B21A70314A50541978C9B242
:10842000481CC0B218700A2050541978C9B2481CB0
:10843000C0B21870002050541C78E4B2611CC9B25C
:1084400019703178C9B24D1CEDB2357011551978DB
:10845000C9B24C1CE4B21C70842454541978C9B2BB
:108460004C1CE4B21C70012454541978C9B20C1984
:10847000E4B21C7050541978C9B2481CC0B21870CC
:108480003E2050541978C9B2481CC0B218701C481C
:108490000468240E54541C78E4B2611CC9B21970EB
:1084A0000168090CC9B211551C78E4B2611CC9B24B
:1084B00019700168090AC9B211551978C9B24C1C62
:1084C000E4B21C700368DBB2535402F00CFFC046E8
:1084D00014080020C005002016020020E806002035
:1084E000CF050020320A0020380A0020FFFFFFFBE2
:1084F00016070020280A00202E0A00206807002006
:10850000E40100200C2A00D130E338D80A2A00D137
:108510005FE301D802F0C2FE0520D24BD24D19789C
:10852000C9B24A1CD2B21A70D04A50541978C9B292
:10853000481CC0B21870042050541978C9B2481CA5
:10854000C0B21870002050541878C0B2411CC9B293
:1085500019702978C9B24C1CE4B22C7011541978E6
:10856000C9B2481CC0B21870882050541978C9B2DA
:10857000481CC0B218700123535402F0B4FE0F2AF5
:1085800001D102F050FE3BD80E2A01D002F0ABFE22
:108590000620B44BB44E1978C9B24A1CD2B21A7034
:1085A000B24A50541978C9B2481CC0B2187005209C
:1085B00050541978C9B2481CC0B2187000205054E9
:1085C0001C78E4B2611CC9B219703178C9B24D1C73
:1085D000EDB2357011551978C9B24C1CE4B21C705B
:1085E000862454541978C9B24C1CE4B21C705054FF
:1085F0001978C9B24C1CE4B21C70505402F073FEDE
:10860000102A00D126E3112A00D18BE302F06BFE81
:10861000382A01D101F010F920D8162A01D102F030
:10862000C0FB09D8142A01D102F0AAFD8D4B01D854
:1086300000F0D5FC02F070FD182A01D100F044FDD5
:1086400001D202F05AFC192A00D11EE11A2A01D0E7
:1086500002F049FE227A00238549FBE0402A01D13D
:1086600002F0DDF944D83A2A01D102F03AF801D2F9
:1086700000F035FD3B2A01D002F035FE0620794B93
:10868000794E1978C9B24A1CD2B21A70774A50543E
:108690001978C9B2481CC0B2187005205054197816
:1086A000C9B2481CC0B21870002050541878C0B22B
:1086B000411CC9B219703178C9B24D1CEDB2357088
:1086C00011541978C9B2481CC0B21870B92050545E
:1086D0001978C9B2481CC0B21870FF2050541978DC
:1086E000C9B2481CC0B21870A379535402F0FBFD04
:1086F000422A01D102F068F801D202F0F3F8432ACD
:1087000001D102F028F8712A01D002F0ECFD04201A
:10871000544B554D1978C9B24A1CD2B21A70534AFB
:1087200050541978C9B2481CC0B218700320505474
:108730001978C9B2481CC0B218700020505418787B
:10874000C0B2411CC9B219702978C9B24C1CE4B23C
:108750002C7011541978C9B2481CC0B21870F1239A
:10876000535402F0C0FD062005243E4B3E4F1978BD
:10877000C9B24A1CD2B21A703C4A50541978C9B2D4
:10878000481CC0B2187054541978C9B2481CC0B201
:108790001870002050541978C9B24D1CEDB21D70EC
:1087A0003D78EDB26E1CF6B23E7055541978C9B2E0
:1087B0004D1CEDB21D70832555541978C9B24D1C5E
:1087C000EDB21D7054541978C9B24C1CE4B21C703F
:1087D000505402F088FD80223368D2021343336084
:1087E00002F081FD3268234B1340336002F07BFDC1
:1087F000052019781C4EC9B24A1CD2B21A701B4A05
:1088000050541978C9B2481CC0B218700420505492
:108810001978C9B2481CC0B218700020505418789A
:10882000C0B2411CC9B219703178C9B24D1CEDB249
:10883000357011541978C9B2481CC0B21870822022
:1088400050541978C9B2481CC0B21870A379535457
:1088500002F049FDD8B282420ED9E018407AC854DD
:108860000133F7E716020020E8060020CF050020BC
:10887000FC060020FFFFFBFF00238B540421EE4A7F
:108880000133E37113680B431360E079002857D07C
:108890000023EA4AD15CD8B2002903D00133182B57
:1088A000F8D11800E64BC41D1978E4B2C9B24A1CCD
:1088B000D2B21A70E34AE44F54541978C9B24C1C2E
:1088C000E4B21C70841DE4B254541C78E4B2611C00
:1088D000C9B21970002111551C78E4B2651CEDB2C3
:1088E0001D703D78EDB26E1CF6B23E7015551C78C9
:1088F000D24EE4B2651CEDB21D70952515551C785D
:10890000E4B2651CEDB21D7011551C78E4B2651C13
:10891000EDB21D70012515551C78E4B26519EDB254
:108920001D701055CCB2844201D302F0DCFC1C78DF
:10893000E4B2651CEDB21D70755C01311555F1E7AF
:108940001324BF4BC04E1978C9B24A1CD2B21A7058
:10895000BC4A54541978C9B24C1CE4B21C7012249D
:1089600054541978C9B24C1CE4B21C7050541C7891
:10897000E4B2611CC9B219703178C9B24D1CEDB2B4
:10898000357011551978C9B24C1CE4B21C7095248D
:1089900054541978C9B24C1CE4B21C705054197864
:1089A000C9B24C1CE4B21C7050541978C9B2481CAE
:1089B000C0B218700C2050541978C9B2481CC0B20B
:1089C00018704D2050541978C9B2481CC0B21870A4
:1089D000752050541978C9B2481CC0B218706C2068
:1089E00050541978C9B2481CC0B218707420505441
:1089F0001978C9B2481CC0B218706920505419784F
:108A0000C9B2481CC0B21870442050541978C9B279
:108A1000481CC0B21870652050541978C9B24C1C5B
:108A2000E4B21C70632454541978C9B24C1CE4B2EB
:108A30001C706F2454541978C9B24C1CE4B21C70D9
:108A4000642454541978C9B24C1CE4B21C705054BC
:108A50001978C9B2481CC0B218707223535402F07E
:108A600042FC07241878784EC0B2411CC9B2197074
:108A700074490C541878C0B2441CE4B21C700A54F7
:108A80001A78D2B2501CC0B21870002088541C78DA
:108A9000E4B2621CD2B21A703278D2B2551CEDB276
:108AA00035700A551A78D2B2541CE4B21C70852471
:108AB0008C541A78D2B2541CE4B21C700E248C541C
:108AC0001A78D2B2541CE4B21C7001248C541A7867
:108AD000D2B21419E4B21C70885402F004FC802253
:108AE00033689202134209D080203268574B1340FA
:108AF000574A336093688343936002E033681343BB
:108B0000336005244E4B504E1878C0B2421CD2B28E
:108B10001A704C4A14541878C0B2441CE4B21C7049
:108B2000042414541878C0B2441CE4B21C7000240D
:108B300014541C78E4B2601CC0B218703078C0B213
:108B4000451CEDB2357010551878C0B2441CE4B223
:108B50001C70872414541878C0B2441CE4B21C70F2
:108B60000B689B03DB0F135402F0BDFB0520344B55
:108B7000354D1978C9B24A1CD2B21A70314A5054D4
:108B80001978C9B2481CC0B2187004205054197822
:108B9000C9B2481CC0B21870002050541878C0B236
:108BA000411CC9B219702978C9B24C1CE4B22C70AE
:108BB00011541978C9B2481CC0B218708B20505497
:108BC0001978C9B2481CC0B21870FF23535402F080
:108BD0008AFB05201A4B1C4D1978C9B24A1CD2B227
:108BE0001A70184A50541978C9B2481CC0B218708B
:108BF000042050541978C9B2481CC0B21870002023
:108C000050541878C0B2411CC9B219702978C9B241
:108C10004C1CE4B22C7011541978C9B2481CC0B273
:108C200018708A2050541978C9B2481CC0B2187004
:108C30008023535402F057FB280A0020FC06002032
:108C400016020020CF050020E8060020FFFFFDFFF0
:108C5000C04000500520C74BC74E1978C9B24A1C06
:108C6000D2B21A70C54A50541978C9B2481CC0B261
:108C70001870042050541978C9B2481CC0B218703A
:108C8000002050541C78E4B2611CC9B219703178CC
:108C9000C9B24D1CEDB2357011551978C9B24C1CD2
:108CA000E4B21C70922454541978C9B24C1CE4B23A
:108CB0001C700B235354B24B187002F014FBA379B1
:108CC000AF4A342B20D00ED82A2B23D005D8282BFE
:108CD0001ED0292B24D1062323E0322B12D0332B94
:108CE0001ED101231DE0FC2B18D005D8362B0DD04A
:108CF0003C2B15D1042314E0FD2B0DD0FE2B0FD1FE
:108D00000A230EE000230CE002230AE0032308E01C
:108D1000052306E0072304E0082302E0092300E01E
:108D200091231370934805260378944CDBB25A1CA8
:108D3000D2B202700622E25403788F4FDBB25A1C83
:108D4000D2B20270E6540378DBB25A1CD2B202707F
:108D50000022E2540378DBB25A1CD2B202703A7895
:108D6000D2B2551CEDB23D70E254854B22001D7805
:108D700003000A2D00D918E1280002F007FE0B00BD
:108D80002400450059006D007B00A400BB00D0000A
:108D9000E50005011978C9B2481CC0B218709020CE
:108DA00060541978C9B2481CC0B21870322060549F
:108DB00074494C310888012800D1BEE00988032994
:108DC00000D0A5E0B9E01878C0B2441CE4B21C7031
:108DD000902414541878C0B2441CE4B21C7033249C
:108DE000145408688021490308401978C9B2002842
:108DF00005D0481CC0B2187001235354EAE04C1C43
:108E0000E4B21C705054E5E01978C9B2481CC0B2F5
:108E10001870902060541978C9B2481CC0B21870FC
:108E20003420605457494C310988022970D884E0B5
:108E30001978C9B2481CC0B21870902060541978D3
:108E4000C9B2481CC0B21870362060544D494C312C
:108E50000988012971D85BE01978C9B2481CC0B2F1
:108E60001870902060541978C9B2481CC0B21870AC
:108E70003C204CE01978C9B2481CC0B21870902050
:108E800060541978C9B2481CC0B2187028206054C8
:108E90003C494C310888012806D81978C9B2481CC9
:108EA000C0B218700423A8E70888022806D11978F0
:108EB000C9B2481CC0B218700C239EE70988022969
:108EC00000D887E039E01978C9B2481CC0B21870E0
:108ED000902060541978C9B2481CC0B2187029207B
:108EE000605428494C31088801285BD90988032936
:108EF0000ED157E01978C9B2481CC0B21870902042
:108F000060541978C9B2481CC0B218702A20505455
:108F10001978C9B2481CC0B2187000236DE71978DF
:108F2000C9B2481CC0B21870902060541978C9B2F8
:108F3000481CC0B21870FD2060541978C9B2481C92
:108F4000C0B21870082358E71978C9B2481CC0B2DB
:108F50001870902060541978C9B2481CC0B21870BB
:108F6000FC2060541978C9B2481CC0B2187018238C
:108F700043E7C04616020020E8060020CF05002087
:108F8000A4010020200200201978C9B2481CC0B2F8
:108F90001870902060541978C9B2481CC0B218707B
:108FA000FE2060541978C9B223E704220378043BF9
:108FB000E6540378033BE2540378DBB25A1CD2B286
:108FC00002709122E2540378DBB25A1CD2B20270D2
:108FD000FF22E254D84B01351D7002F084F90620BF
:108FE0001978D64EC9B24A1CD2B21A70D44A50541B
:108FF0001978C9B2481CC0B21870052050541978AD
:10900000C9B2481CC0B21870002050541878C0B2C1
:10901000411CC9B219703178C9B24D1CEDB235701E
:1090200011541978C9B2481CC0B21870902050541D
:109030001978C9B2481CC0B21870A07950543328AE
:109040001DD1E479BF49002C0DD080240868640349
:10905000204308601978C9B2481CC0B218700123B7
:10906000535402F040F90D68B74828400860197859
:10907000C9B2481CC0B21870545402F034F92928FF
:1090800019D1B2494C310888012802D9098803292D
:1090900008D11978C9B2481CC0B2187001235354C2
:1090A00002F021F91978C9B2481CC0B21870002327
:1090B000535402F018F91978C9B2481CC0B218709C
:1090C0000023535402F00FF9A279A14B1A70E279F0
:1090D0005A70227A9A70627ADA7002F004F99D4B23
:1090E000974D1A78954ED2B2511CC9B21970092108
:1090F000A9541A78D2B2511CC9B219700821A954C6
:109100001A78D2B2511CC9B219700021A954197829
:10911000C9B24A1CD2B21A703278D2B2501CC0B254
:1091200030706A541A78D2B2511CC9B21970B82181
:10913000A9541978C9B24A1CD2B21A70A2796A54D9
:109140000B2A01D902F0CFF8100002F01FFC0C002E
:1091500014001C0024006500C3003D019B01F901BF
:109160004F02A4021F0379494C310988022902D910
:109170000422A27158E075494C310988022902D9AC
:109180000432A271AEE071494C310988022902D93A
:109190000432A27120E16D4908004C300088022899
:1091A00002D90432A27175E10126520096403200C4
:1091B0001878C0B2441CE4B21C70674C247822407A
:1091C00054426241D2B22A541878C0B2421CD2B280
:1091D0001A7002222A5461480068C00607D51A781E
:1091E000D2B2511CC9B219708021A9540BE0187871
:1091F0008431C0B2441CE4B21C7009880A40514258
:109200004A4152002A541A78D2B2511CC9B219707C
:109210000023AB5402F067F84C4A4C321288022A01
:1092200002D90822A2718BE14D4A117801220A402D
:10923000A179022404390A411978D2B2C9B2481C72
:10924000C0B218706A541A78D2B2511CC9B21970DF
:10925000AC54424A1168202211400FD01A78D2B281
:10926000511CC9B219708021A9541A78D2B2511C6C
:10927000C9B219700023AB5402F035F839483A4EA0
:1092800007883288974217D01A78D2B2511CC9B2D7
:1092900019700321A9541C78E4B2621CD2B21A706E
:1092A000324B008831881A8880B289B292B2F7F7BF
:1092B000BDFD285502F017F81A78D2B2501CC0B282
:1092C0001870AC541A78D2B2501CC0B21870A9549D
:1092D00002F009F81D4A4C321288022A02D90922EA
:1092E000A27183E102211E4AA079127804380A4053
:1092F00002411878D2B2C0B2441CE4B21C702A54A5
:109300001A78D2B2501CC0B21870A954134A10680F
:10931000202210402CD01A78D2B2511CC9B2197038
:109320008021A9541A78D2B2511CC9B219700023F5
:10933000AB5401F0D8FFC046A4010020E80600208D
:10934000CF05002068070020FFFFEFFF200200206C
:10935000120200201602002090040020200A0020A3
:10936000E9060020E406002078040020340A0020EA
:10937000DE4FDF4E3C883288944217D01A78D2B242
:10938000511CC9B219700321A9541C78E4B2621CA3
:10939000D2B21A70D74B388831881A8880B289B215
:1093A00092B2F7F743FD285501F09DFF1A78D2B22B
:1093B000541CE4B21C70A9541A78D2B2511CC9B220
:1093C0001970A85401F08FFFCB4A4C321288022A40
:1093D00002D90A22A2715EE1C84A117804220A4029
:1093E000A179022404390A411978D2B2C9B2481CC1
:1093F000C0B218706A541A78D2B2511CC9B219702E
:10940000AC54BF4A1168202211400FD01A78D2B252
:10941000511CC9B219708021A9541A78D2B2511CBA
:10942000C9B219700023AB5401F05DFFB548B64EC8
:1094300007883288974217D01A78D2B2511CC9B225
:1094400019700321A9541C78E4B2621CD2B21A70BC
:10945000AE4B008831881A8880B289B292B2F7F791
:10946000E5FC285501F03FFF1A78D2B2501CC0B27B
:109470001870AC541A78D2B2501CC0B21870A954EB
:1094800001F031FF9C4A4C321288022A02D90B2289
:10949000A2717BE1994A117808220A40A17902243D
:1094A00004390A411978D2B2C9B2481CC0B2187046
:1094B0006A541A78D2B2511CC9B21970AC54904A8D
:1094C0001168202211400FD01A78D2B2511CC9B2B3
:1094D00019708021A9541A78D2B2511CC9B21970DE
:1094E0000023AB5401F0FFFE89488A4E078832887A
:1094F000974217D01A78D2B2511CC9B21970032101
:10950000A9541C78E4B2621CD2B21A70824B008853
:1095100031881A8880B289B292B2F7F787FC285551
:1095200001F0E1FE1A78D2B2501CC0B21870AC54EF
:109530001A78D2B2501CC0B21870A95401F0D3FEF0
:109540006E4A117810220A40A179022404390A4196
:109550001978D2B2C9B2481CC0B218706A541A78CD
:10956000D2B2511CC9B21970AC54654A116820229C
:1095700011400FD01A78D2B2511CC9B21970802193
:10958000A9541A78D2B2511CC9B219700023AB5435
:1095900001F0A9FE6148624E07883288974217D0D1
:1095A0001A78D2B2511CC9B219700321A9541C787F
:1095B000E4B2621CD2B21A705A4B008831881A8801
:1095C00080B289B292B2F7F731FC285501F08BFED8
:1095D0001A78D2B2501CC0B21870AC541A78D2B2F9
:1095E000501CC0B21870A95401F07DFE2021434ADE
:1095F000A079127804380A4002411878D2B2C0B279
:10960000441CE4B21C702A541A78D2B2501CC0B266
:1096100018700220A8543A4A126811400FD01A78E4
:10962000D2B2511CC9B219708021A9541A78D2B291
:10963000511CC9B219700023AB5401F054FE3A4FCB
:109640003A4E3C883288944217D01A78D2B2511CD4
:10965000C9B219700321A9541C78E4B2621CD2B2B9
:109660001A70334B388831881A8880B289B292B226
:10967000F7F7DCFB285501F036FE1A78D2B2541CFD
:10968000E4B21C70A8541A78D2B2501CC0B2187040
:10969000A95401F028FE194A117840220A40A17904
:1096A000022404390A411978D2B2C9B2481CC0B2A6
:1096B00018706A541A78D2B2511CC9B21970AC54DD
:1096C0000F4A11682022114034D01A78D2B2511CAE
:1096D000C9B219708021A9541A78D2B2511CC9B2EA
:1096E00019700023AB5401F0FEFDC0467A0400203F
:1096F000F60600206207002020020020E906002074
:10970000200A002098040020180A0020B604002037
:10971000660700209E040020B40400200002002000
:10972000100200201008002058070020020200202C
:109730007E040020D748D84E07883288974217D039
:109740001A78D2B2511CC9B219700321A9541C78DD
:10975000E4B2621CD2B21A70D04B008831881A88E9
:1097600080B289B292B2F7F761FB285501F0BBFDD8
:109770001A78D2B2501CC0B21870AC541A78D2B257
:10978000501CC0B21870A95401F0ADFD7F21C44A2D
:1097900012788A43A179022404390A411978D2B295
:1097A000C9B2481CC0B218706A541A78D2B2511C9F
:1097B000C9B21970AC54BB4A1168202211400FD0B5
:1097C0001A78D2B2511CC9B219708021A9541A78E2
:1097D000D2B2511CC9B219700023AB5401F083FD01
:1097E000B148B24E07883288974217D01A78D2B261
:1097F000511CC9B219700321A9541C78E4B2621C2F
:10980000D2B21A70AA4B008831881A8880B289B205
:1098100092B2F7F70BFB285501F065FD1A78D2B22A
:10982000501CC0B21870AC541A78D2B2501CC0B2DE
:109830001870A95401F057FD9E4B9F4D1A789F4E0A
:10984000D2B2511CC9B219700921A9541A78D2B2E6
:10985000511CC9B219700821A9541A78D2B2511CEE
:10986000C9B219700021A9541978C9B24A1CD2B2E0
:109870001A703278D2B2501CC0B230706A541A7862
:10988000D2B2511CC9B21970B821A9541A78D2B2F7
:10989000511CC9B21970A079A8541978C9B24A1CD0
:1098A000D2B21A70E2796A541978C9B24C1CE4B287
:1098B0001C7002246C540B2801D901F014FD804C5B
:1098C00021004C3102F062F80C00B1007D0126024B
:1098D000EA026A03EA036A0405058005FB059106AE
:1098E0000988022900D9DDE276497748002A4ED05E
:1098F00010278268754E3A4382608268FF19BA4326
:109900008260642220894243714892B202806F4A89
:1099100010780222104330700878104214D0187862
:109920008434C0B2411CC9B2197021880A40514226
:109930004A4152002A541A78D2B2511CC9B2197045
:109940000023AB5401F0CFFC0878024301200A70D9
:109950000A7882430A701A78D2B21118C9B2197003
:10996000A85422893F2A09D81A78D2B21118C9B24C
:1099700019702389DBB2AB5401F0B5FC1A78D2B26E
:10998000511CC9B219703F23AB5401F0ACFC202626
:109990008768374387608768103EB74387606420D5
:1099A000E7884A4E78434B4F80B2388001274748BA
:1099B0000078384330700878384213D018788434EF
:1099C000C0B2C119C9B21970218839404C426141F5
:1099D000B94029541978C9B2C819C0B218706A546C
:1099E00001F081FC02200A783A430A700A78824327
:1099F0000A701A78D2B2511CC9B21970AF54E288F9
:109A00003F2A09D81A78D2B2511CC9B21970E3881A
:109A1000DBB2AB5401F067FC1A78D2B2511CC9B268
:109A200019703F23AB5401F05EFC0988022900D96C
:109A3000B8E224492448002A74D040278268234E83
:109A40003A4382608268FF19BA4382601F4A1078E5
:109A50000822104330706420A68970431E4E80B2E5
:109A600030800878104239D018788434C0B2411C54
:109A7000C9B2197021880A4051424A4152002A5401
:109A80001A78D2B2511CC9B219700023AB5401F03C
:109A90002AFCC04680040020F4060020300A002082
:109AA000E9060020200A0020FA0600207C0400209D
:109AB000160A002016020020CF050020E80600202C
:109AC0002002002090040020004100506007002088
:109AD000820400209A040020E60600200878024351
:109AE00004200A700A7882430A701A78D2B2511C94
:109AF000C9B219700121A954A2893F2A09D81A783C
:109B0000D2B25118C9B21970A389DBB2AB5401F0BB
:109B1000EAFB1A78D2B2511CC9B219703F23AB5478
:109B200001F0E1FB80268768374387608768403E05
:109B3000B743876064206789D04E7843D04F80B2A6
:109B400038800427CD480078384330700878384290
:109B500013D018788434C0B2411CC9B2197021885E
:109B600039404C426141490029541978C9B2481C16
:109B7000C0B218706A5401F0B6FB08200A78174387
:109B80000F700A7882430A701A78D2B2511CC9B297
:109B900019700121A95462893F2A09D81A78D2B2D2
:109BA0005118C9B219706389DBB2AB5401F09BFB49
:109BB0001A78D2B2511CC9B219703F23AB5401F0CC
:109BC00092FB0988022900D96CE2AE49002A4FD0E5
:109BD000012002268A68A94F02438A608A68B2433C
:109BE0008A606422A11DCE8F7243A74E92B232804A
:109BF00020223E7816433E70A44E3778174214D088
:109C000018788434C0B2411CC9B2197021880A4046
:109C100051424A4152002A541A78D2B2511CC9B258
:109C200019700023AB5401F05EFB347822431024FA
:109C300032703278A24332701A78D2B2541CE4B235
:109C40001C70A854CA8F3F2A09D81A78D2B2501C67
:109C5000C0B21870CB8FDBB2AB5401F044FB1A7862
:109C6000D2B2511CC9B219703F23AB5401F03BFB77
:109C700002268868304388608868013EB043886067
:109C80006421261DF08F4143814889B201807B49C0
:109C900010208C4667460978014339707B490F785C
:109CA000074213D019788434C9B24E1CF6B21E7024
:109CB0002488204044426041400068541978C9B269
:109CC000481CC0B218706A5401F00DFB0A781043AA
:109CD000087020200A7882430A701A78D2B2511C88
:109CE000C9B219700121A954F28F3F2A09D81A78F4
:109CF000D2B2511CC9B21970F38FDBB2AB5401F070
:109D0000F2FA1A78D2B2511CC9B219703F23AB547F
:109D100001F0E9FA0988022900D943E25B49594870
:109D2000002A55D0042682688027324382608268E8
:109D3000B619B243826020006422483006887F4210
:109D40007243544E92B232804C4A16783E43F6B279
:109D500016700A7852B2002A15DA19788434C9B21A
:109D60004A1CD2B21A7080222088024050424241DE
:109D700052006A541A78D2B2511CC9B21970002329
:109D8000AB5401F0B0FA40240A783A43D2B20A70D8
:109D90000A78A2430A701A78D2B2511CC9B219705B
:109DA0000121A95402883F2A09D81A78D2B2511841
:109DB000C9B219700388DBB2AB5401F094FA1A7877
:109DC000D2B2511CC9B219703F23AB5401F08BFAC7
:109DD000082786683E4386608668043FBE438660E7
:109DE0002600642008360196F78F78432A4F80B208
:109DF00038802248844607784020664607433770FB
:109E00000F78074213D019788434C9B24E1CF6B2C9
:109E10001E702488204044426041400068541978F4
:109E2000C9B2481CC0B218706A5401F05CFA0A78D2
:109E300010437F220870087802400A701A78D2B264
:109E4000511CC9B219700121A954019AD28F3F2A1D
:109E50000AD81A78D2B25118C9B21970019BDB8F97
:109E6000DBB2AB5401F03FFA1A78D2B2511CC9B23E
:109E700019703F23AB5401F036FAC046600700204A
:109E80008A040020004100501208002090040020A5
:109E9000EC060020140700205E0700200888022836
:109EA00000D075E0D149002A39D022005032108804
:109EB0000A88904219D11A78D2B2511CC9B21970CD
:109EC0000321A9541E78F6B2721CD2B21A70230074
:109ED00052331888C64B80B21988C64B89B21A888B
:109EE00092B2F6F7A3FFA8550DE01A78D2B2511C32
:109EF000C9B219700221A9541A78D2B2511CC9B240
:109F000019700023AB54012152342388B74A9BB205
:109F10001380B94A13780B43137001F0E4F9200061
:109F2000523000880988884219D11A78D2B2511C5F
:109F3000C9B219700321A9541E78F6B2721CD2B2AC
:109F40001A70230050331888A94B80B21988A94B86
:109F500089B21A8892B2F6F769FFA8550CE0197811
:109F6000C9B2481CC0B21870022068541978C9B22E
:109F7000481CC0B218706A540121503423889B4A8F
:109F80009BB213809C4A13788B43137001F0ABF99A
:109F90000988022900D9A1E101F0A5F90888022861
:109FA00000D075E09549002A39D022005632108839
:109FB0000A88904219D11A78D2B2511CC9B21970CC
:109FC0000321A9541E78F6B2721CD2B21A70230073
:109FD000583318888A4B80B219888A4B89B21A88FC
:109FE00092B2F6F723FFA8550DE01A78D2B2511CB1
:109FF000C9B219700221A9541A78D2B2511CC9B23F
:10A0000019700023AB540221583423887B4A9BB239
:10A010001380794A13780B43137001F064F9200020
:10A02000583000880988884219D11A78D2B2511C58
:10A03000C9B219700321A9541E78F6B2721CD2B2AB
:10A040001A702300563318886D4B80B219886D4BF7
:10A0500089B21A8892B2F6F7E9FEA8550CE0197891
:10A06000C9B2481CC0B21870022068541978C9B22D
:10A07000481CC0B218706A540221563423885F4AC3
:10A080009BB213805C4A13788B43137001F02BF959
:10A090000988022900D99CE101F025F908880228E5
:10A0A00000D075E05849002A39D022005C3210886F
:10A0B0000A88904219D11A78D2B2511CC9B21970CB
:10A0C0000321A9541E78F6B2721CD2B21A70230072
:10A0D0005E3318884D4B80B219884D4B89B21A886F
:10A0E00092B2F6F7A3FEA8550DE01A78D2B2511C31
:10A0F000C9B219700221A9541A78D2B2511CC9B23E
:10A1000019700023AB5404215E3423883E4A9BB26D
:10A110001380394A13780B43137001F0E4F82000E0
:10A120005E3000880988884219D11A78D2B2511C51
:10A13000C9B219700321A9541E78F6B2721CD2B2AA
:10A140001A7023005C331888304B80B21988304B6A
:10A1500089B21A8892B2F6F769FEA8550CE0197810
:10A16000C9B2481CC0B21870022068541978C9B22C
:10A17000481CC0B218706A5404215C342388224AF7
:10A180009BB213801C4A13788B43137001F0ABF819
:10A190000988022900D997E101F0A5F8088802286A
:10A1A00000D090E01B49002A54D02200623210886F
:10A1B0000A88904234D11A78D2B2511CC9B21970AF
:10A1C0000321A9541E78F6B2721CD2B21A70230071
:10A1D00064331888104B80B21988104B89B21A88E2
:10A1E00092B2F6F723FEA85528E0C046E406002008
:10A1F00078040020340A0020E90600207A040020B8
:10A20000F60600206207002098040020180A0020AB
:10A21000B6040020660700209E040020B40400203D
:10A220001A78D2B2511CC9B219700221A9541A78F5
:10A23000D2B2511CC9B219700023AB540821643446
:10A240002388D04A9BB21380CF4A13780B431370F4
:10A2500001F049F82000643000880988884219D14B
:10A260001A78D2B2511CC9B219700321A9541E78B0
:10A27000F6B2721CD2B21A70230062331888C34B34
:10A2800080B21988C24B89B21A8892B2F6F7CEFD15
:10A29000A8550CE01978C9B2481CC0B21870022049
:10A2A00068541978C9B2481CC0B218706A540821A1
:10A2B00062342388B34A9BB21380B34A13788B432A
:10A2C000137001F010F80988022900D992E101F019
:10A2D0000AF80988022901D001F005F8AD49002AE1
:10A2E00039D02200683210880A88904219D11A7831
:10A2F000D2B2511CC9B219700321A9541E78F6B20A
:10A30000721CD2B21A7023006A331888A24B80B232
:10A310001988A24B89B21A8892B2F6F787FDA85520
:10A320000DE01A78D2B2511CC9B219700221A95499
:10A330001A78D2B2511CC9B219700023AB54102143
:10A340006A342388934A9BB213808F4A13780B4355
:10A35000137000F0C8FF20006A3000880988884226
:10A3600019D11A78D2B2511CC9B219700321A9545B
:10A370001E78F6B2721CD2B21A70230068331888A5
:10A38000854B80B21988854B89B21A8892B2F6F74C
:10A390004DFDA8550CE01978C9B2481CC0B2187020
:10A3A000022068541978C9B2481CC0B218706A54A7
:10A3B000102168342388774A9BB21380724A13783D
:10A3C0008B43137000F08FFF0988022901D000F041
:10A3D0008AFF7349002A39D022006E3210880A8819
:10A3E000904219D11A78D2B2511CC9B21970032106
:10A3F000A9541E78F6B2721CD2B21A7023007033C0
:10A400001888684B80B21988674B89B21A8892B253
:10A41000F6F70CFDA8550DE01A78D2B2511CC9B25E
:10A4200019700221A9541A78D2B2511CC9B21970FC
:10A430000023AB54202170342388594A9BB21380E7
:10A44000514A13780B43137000F04DFF2000703019
:10A4500000880988884219D11A78D2B2511CC9B231
:10A4600019700321A9541E78F6B2721CD2B21A7068
:10A4700023006E3318884B4B80B219884A4B89B23F
:10A480001A8892B2F6F7D2FCA8550CE01978C9B236
:10A49000481CC0B21870022068541978C9B2481C10
:10A4A000C0B218706A5420216E3423883C4A9BB293
:10A4B0001380354A13788B43137000F014FF09881A
:10A4C000022901D000F00FFF3849002A39D02200BC
:10A4D000743210880A88904219D11A78D2B2511C6D
:10A4E000C9B219700321A9541E78F6B2721CD2B2F7
:10A4F0001A702300763318882D4B80B219882D4BA3
:10A5000089B21A8892B2F6F791FCA8550DE01A7834
:10A51000D2B2511CC9B219700221A9541A78D2B210
:10A52000511CC9B219700023AB54402176342388E2
:10A530001E4A9BB21380144A13780B43137000F029
:10A54000D2FE2000763000880988884234D11A78FB
:10A55000D2B2511CC9B219700321A9541E78F6B2A7
:10A56000721CD2B21A70230074331888104B80B258
:10A570001988104B89B21A8892B2F6F757FCA85581
:10A5800027E0C04666070020E90600209E04002060
:10A59000B404002000020020100200201008002057
:10A5A00058070020020200207E04002080040020C2
:10A5B000F4060020300A00201978C9B2481CC0B245
:10A5C0001870022068541978C9B2481CC0B21870BB
:10A5D0006A54402174342388B94A9BB21380B94A23
:10A5E00013788B43137000F07EFE0988022901D096
:10A5F00000F079FEB449002A3AD022007A3210885D
:10A600000A88904219D11A78D2B2511CC9B2197075
:10A610000321A9541E78F6B2721CD2B21A7023001C
:10A620007C331888A94B80B21988A94B89B21A8843
:10A6300092B2F6F7FBFBA8550DE01A78D2B2511C86
:10A64000C9B219700221A9541A78D2B2511CC9B2E8
:10A6500019700023AB5480217C3423889A4A9BB222
:10A660001380984A494213780B43137000F03BFE65
:10A6700020007C3000880988884219D11A78D2B22B
:10A68000511CC9B219700321A9541E78F6B2721C6C
:10A69000D2B21A7023007A3318888C4B80B2198892
:10A6A0008B4B89B21A8892B2F6F7C0FBA8550CE022
:10A6B0001978C9B2481CC0B21870022068541978C1
:10A6C000C9B2481CC0B218706A547A3423887E4AD2
:10A6D0009BB213807F237B4A11780B40137000F0EC
:10A6E00002FE06207B4B7C4E1978C9B24A1CD2B2BE
:10A6F0001A707A4A50541978C9B2481CC0B21870FE
:10A70000052050541978C9B2481CC0B218700020F6
:10A7100050541878C0B2411CC9B219703178C9B20E
:10A720004D1CEDB2357011541978C9B2481CC0B235
:10A730001870B92050541978C9B2481CC0B21870AA
:10A74000FF2050541978C9B2481CC0B21870A379C0
:10A75000535400F0C8FD06205E4B5F4F1978C9B214
:10A760004A1CD2B21A705D4A50541978C9B2481CBA
:10A77000C0B21870052050541978C9B2481CC0B234
:10A780001870002050541978C9B24D1CEDB21D70DC
:10A790003D78EDB26E1CF6B23E7055541978C9B2D0
:10A7A0004D1CEDB21D70C32555541978C9B24D1C0E
:10A7B000EDB21D70A47954541978C9B24C1CE4B29E
:10A7C0001C70505400F08FFDA379022B00D0AFE233
:10A7D000434B4C331B88012B00D8A9E2E279072AAE
:10A7E00000D9A5E23B4C3D4D23783B4EDBB2591CD2
:10A7F000C9B221700A21E9542378DBB2591CC9B2CD
:10A8000021700921E9542378DBB2591CC9B22170A7
:10A810000021E9542378DBB2591CC9B22170317888
:10A82000C9B2481CC0B23070E95423780326DBB2A9
:10A83000591CC9B22170C221E95423785643DBB2B6
:10A84000591CC9B221700221E9542378DBB2591C8A
:10A85000C9B22170EA542778214AFFB27B1CDBB2CF
:10A860002370330028335B00985A642180B201F0D2
:10A8700097F8C0B2E8552778194AFFB27B1CDBB2C3
:10A880002370330029335B00985A642180B201F0B1
:10A8900087F8C0B2E85523782A36DBB25A1CD2B208
:10A8A00022700F4A7600B25AD2B2EA542378DBB251
:10A8B0005A1CD2B222700022EA5400F014FDC046A5
:10A8C00080040020E9060020FA0600207C04002015
:10A8D000160A002016020020E8060020CF050020FE
:10A8E00020020020D54B4C331B88012B00D81FE2DF
:10A8F000A3790293022B00D01AE2E3790193072B8C
:10A9000000D915E203255D43EFB238006423217AB4
:10A9100028305943C0B2F6F733F92B00C74E28331D
:10A920005B009853380003936423617A29305943BC
:10A93000C0B2F6F725F92B0029335B009853049336
:10A940002A37A17AF8B2F6F71BF92A35BC4C6B000E
:10A95000985305932378BB4DDBB25A1CD2B22270B8
:10A960000A22EA542378B848DBB25A1CD2B22270C9
:10A970000922EA542378DBB25A1CD2B22270002298
:10A98000EA542278D2B2531CDBB223700378DBB2D4
:10A99000591CC9B20170AB5423786421DBB25A1C34
:10A9A000D2B22270C222EA542378DBB25A1CD2B24D
:10A9B00022706A46127AEA542378DBB25A1CD2B269
:10A9C00022706A461279EA542778FFB27B1CDBB208
:10A9D0002370039B985B80B200F0E2FFC0B2E855A1
:10A9E00027786421FFB27B1CDBB22370049B985B49
:10A9F00080B200F0D5FFC0B2E8552378DBB25A1C14
:10AA0000D2B22270059A925BD2B2EA542378DBB2BA
:10AA10005A1CD2B222700022EA5400F064FCA079E1
:10AA2000874B002803D0022800D113E180E1834A3C
:10AA300011004C310988022900D979E1E17907290F
:10AA400000D975E1080000F097FF041A30465C73E6
:10AA50008AA2D288002A00D06AE1247A20257B4885
:10AA60007B4A002C05D084682C4384601078012434
:10AA70009DE08468AC4384601078012485E01289ED
:10AA8000002A00D054E1247A10257048704A002C26
:10AA900005D084682C4384601078022487E08468A1
:10AAA000AC438460107802246FE05289002A00D001
:10AAB0003EE1247A80256548654A002C05D08468EB
:10AAC0002C4384601078042471E08468AC43846073
:10AAD0001078042459E09289002A00D028E1247AD1
:10AAE00040255A485A4A002C05D084682C4384607B
:10AAF000107808245BE08468AC43846010780824F4
:10AB000043E00432D28F002A00D011E1247A0225DA
:10AB10004E484F4A002C05D084682C43846010783E
:10AB2000102444E08468AC438460107810242CE046
:10AB30000632D28F002A00D0FAE0247A0125434859
:10AB4000434A002C05D084682C438460107820246C
:10AB50002DE08468AC4384601078202415E008322E
:10AB6000D28F002A00D0E3E0247A08253748384AFB
:10AB7000002C05D084682C4384601078402416E0B3
:10AB80008468AC43846040241078A04317E04832C6
:10AB90001288002A00D0CBE0247A04252B482C4AC6
:10ABA000002C06D084682C438460802014782043D5
:10ABB00005E08468AC4384607F201478204007243B
:10ABC00010701878204FC0B2421CD2B21A701D4AC1
:10ABD00014541878C0B2441CE4B21C7006241454F7
:10ABE0001878C0B2441CE4B21C70002414541878C5
:10ABF000C0B2451CEDB21D703D78EDB26E1CF6B2D0
:10AC00003E7015541878C0B2451CEDB21D70C025B9
:10AC100015541878C0B2451CEDB21D701454187844
:10AC2000C0B2441CE4B21C7011541978C9B2481C5B
:10AC3000C0B2187006AB1B7A535454E320020020B4
:10AC400016020020CF050020E80600200041005039
:10AC500060070020DD4A4C321288012A68D9072596
:10AC60001978DB4FC9B24A1CD2B21A70D94A55546E
:10AC70001978C9B24D1CEDB21D70062555541978CE
:10AC8000C9B24D1CEDB21D70002555541978C9B2DA
:10AC90004D1CEDB21D703D78EDB26E1CF6B23E70EB
:10ACA00055541978C9B24D1CEDB21D70C0255554CC
:10ACB0001978C9B24D1CEDB21D7050541978C9B243
:10ACC000481CC0B21870E57955541978C9B2481CAF
:10ACD000C0B21870FA23207ADB0050545843FF2189
:10ACE00000F0E8FE0300F533FF339BB2072D00D9D7
:10ACF000F9E2280000F040FE04070A0D10131619AF
:10AD0000B54A1380EFE2B54A1380ECE2B44A1380EF
:10AD1000E9E2B44A1380E6E2B34A1380E3E2B34ABD
:10AD20001380E0E2B24A1380DDE2B24A1380DAE235
:10AD30000620B14BA64E1978C9B24A1CD2B21A707D
:10AD4000A44A50541978C9B2481CC0B218700520E2
:10AD500050541978C9B2481CC0B218700020505421
:10AD60001878C0B2411CC9B219703178C9B24D1CF3
:10AD7000EDB2357011541978C9B2481CC0B21870C0
:10AD8000C12050541978C9B2481CC0B21870E0797B
:10AD900050541978C9B2481CC0B21870237A535461
:10ADA000A1E2A179092903D86318D879092808D91B
:10ADB0003268924B134033603268914B13403360DA
:10ADC0000DE38D4B0D181E78EDB2F6B2721CD2B2A7
:10ADD0001A70AF1D7F4AFFB297551E780535F6B23F
:10ADE000771CFFB2EDB21F7095551D78EDB26E1C49
:10ADF000F6B21E70002656551D78EDB26E1CF6B2E6
:10AE00001E70734E0195B44665463678F6B2771CCF
:10AE1000FFB22F70019D56551D78EDB26E1CF6B233
:10AE20001E70932656551D78EDB26E1CF6B21E703C
:10AE300051550025EEB2B14209D91E78F6B2771C01
:10AE4000FFB21F706719FF7901359755F2E71C783B
:10AE5000E4B2651CEDB21D7010550024E5B2A842A5
:10AE60000BD91D7806AFEDB26E1CF6B21E706618D7
:10AE7000F619367A01345655F0E700220A2406AB5B
:10AE8000DD79303DEDB20132D3B2994207D906AE39
:10AE900065439319DB79303BED18EDB2F3E706AA71
:10AEA0008B180A2600221C7A303CE4B20132D3B25D
:10AEB000984208D9531806AF7443DB191B7A303B0C
:10AEC000E418E4B2F2E76E1EA7B2F6B23900300021
:10AED000F5F78EFE874203D039003000F5F788FE83
:10AEE000072D00D0FFE13E2C00D0FCE18021454A37
:10AEF000090513680B431360F5E1A279092A08D903
:10AF000032683E4B1340336032683D4B1340336030
:10AF100065E200200A25E379303BDFB20130C3B29D
:10AF20009A4208D93E002318D9796E430B00303B72
:10AF3000F318DFB2F2E7072F03D18721234B490033
:10AF4000D9812D4C234D2378DBB2591CC9B2217015
:10AF500011000931C9B2E9542378DBB2591CC9B2D6
:10AF6000217011000831C9B2E9542178C9B24B1CD3
:10AF7000DBB2237000236B542178C9B2481CC0B2E5
:10AF800020701348844663460078C0B2461CF6B26F
:10AF90001E70685420780023C0B2411CC9B22170D1
:10AFA000932129542178C9B2481CC0B220706A5438
:10AFB000D9B2914228D2207806AEC0B2411CC9B2A3
:10AFC00021709919C97901332954F1E72002002031
:10AFD000E8060020CF050020E40600207A040020C7
:10AFE0009804002066070020000200205807002077
:10AFF00080040020FA06002016020020FFFFFFFD5B
:10B00000FFFFFFFB680700202378E04EDBB25A1CED
:10B01000D2B222700322EA543B00283B172B54D9AA
:10B020008B2F19D87B00F25AD2B2F252012F03D1E2
:10B030006F22F15A0A40F25222786421D2B2019270
:10B040000132D2B22270F05A80B200F0A9FC019B0A
:10B050003030C0B2E8543FE03B00643B5B00F05A44
:10B0600027780193FFB27B1CDBB22370642180B28E
:10B0700000F096FC6421C0B200F092FC3030019BDD
:10B08000C0B2E855F05A642180B200F089FC642116
:10B09000C0B200F00BFD2678CFB2F6B2731CDBB263
:10B0A00023700A21380000F07BFC3030C0B2A85574
:10B0B00026780A21F6B2731CDBB22370380000F048
:10B0C000F5FC3031C9B2A9550DE12378DBB25A1C29
:10B0D000D2B222703022EA547B00F05A642180B24E
:10B0E00000F0E4FC2678CFB2F6B2731CDBB223701A
:10B0F0000A21380000F054FC3030C0B2A855267840
:10B100000A21F6B2731CDBB22370380000F0CEFCCB
:10B110003031C9B2A955E6E0052031689C4A0A40A1
:10B12000326019789B4EC9B24A1CD2B21A709A4A40
:10B1300050541978C9B2481CC0B218700420505439
:10B140001978C9B2481CC0B21870002050541C783D
:10B15000E4B2611CC9B219703178C9B24D1CEDB2AC
:10B16000357011551978C9B24C1CE4B21C70942486
:10B1700054541978C9B24C1CE4B21C705054B2E05B
:10B18000864B607A1A68120E904200D0ABE01A68C3
:10B19000A07A120CD2B2904200D0A4E0FF201A682C
:10B1A000E57A120A0240954200D09CE01B68227B9F
:10B1B00003409A4200D096E0802233689204134301
:10B1C0003360774BFA381978724DC9B24A1CD2B243
:10B1D0001A70714A50541978C9B2481CC0B218701C
:10B1E000042050541978C9B2481CC0B2187000200D
:10B1F00050541878C0B2411CC9B219702978C9B22C
:10B200004C1CE4B22C7011541978C9B2481CC0B25D
:10B210001870942050541978C9B2481CC0B21870E4
:10B22000012353545FE0A379002B5CD1637A3E2B5A
:10B2300059D15A49A27A0B681B0E9A4253D1FF2367
:10B240000A68E07A120C1A4090424CD10A68207BBE
:10B25000120A1A40904246D10968627B0B409A421A
:10B2600041D1F5F77FFCF5F765FCF8204002F5F7D2
:10B2700037FC2B784B4A4C4C1B021343236021684C
:10B280004A48F5F7D3FB0321494A13680B4323606F
:10B2900023681360474A484B1A60FEE78022474BF9
:10B2A0009201DA670022464BFF211A70FA22454BC1
:10B2B000D2001A80444A11701A0013889BB2002BE6
:10B2C000FBD1344A1370F5F74DFC0321384A13685B
:10B2D0000B431360374A384B02391A60A022D2055B
:10B2E00093680B43936006AB9A78002A36D11B799A
:10B2F000042B2ED0092B07D0032B2FD18021334ACA
:10B30000C90213680B4328E080212C4B8901D967BF
:10B310002B4BFF211A70FA222A4BD2001A802A4A9C
:10B3200011701A0013889BB2002BFBD1194A1370BD
:10B33000F5F718FC03211E4A13680B4313601D4ADE
:10B340001D4B02391A60A022D20593680B4393600B
:10B3500004E01E4A1E4B11680B40136006AB1A78BE
:10B360005B7801339A4235DDDBB2D21A06A90A7046
:10B37000002201320098D1B2884201D8FCF7B8FF10
:10B3800006A81918895C8154F3E7C0462002002002
:10B39000FFFFFFFDE8060020CF050020E4010020AC
:10B3A000160200203E00FFFFFC0100201CF00100FF
:10B3B00000C000500400FA050CED00E004E100E0DC
:10B3C0003D0A00205C070020C1050020680700201E
:10B3D000FFFFFBFF034A044B11680B40136017B0DB
:10B3E000F0BDC04668070020FFFFFFFBF7B5684BC4
:10B3F0001A5C8A4200D1C9E0664A1478002C00D059
:10B40000C4E06434147080221954634B92041D68A4
:10B41000154000D0BAE01A68520300D4B6E0802488
:10B420001A68E40422431A600723034001930029A9
:10B430006DD00126330083400F27DBB20093574BBA
:10B440001C78E4B2A219D2B21A70554A17551C786A
:10B45000E4B2A719FFB21F70082717551C78E4B291
:10B46000A719FFB21F7015551C78E4B2A519EDB2EB
:10B470001D704C4DAC4660462D78EDB2AF19FFB251
:10B48000077015551C786846E4B2A519EDB21D7019
:10B49000BA2515551C780079E4B2A519EDB21D70D6
:10B4A0001055414C4C342488022C08D93F4C00984C
:10B4B000247820400FD01878C0B2841907E03C4CA3
:10B4C00000982478204006D01878C0B2441CE4B21A
:10B4D0001C70165405E01C78E4B2651CEDB21D70BA
:10B4E00010551878C0B2441CE4B21C7002241454E5
:10B4F0001878C0B2441CE4B21C708024145418782C
:10B50000C0B2441CE4B21C700723135408E0234863
:10B510000378DBB25A1CD2B202700620204AD05403
:10B5200005241E4B1F4E1878C0B2421CD2B21A70AE
:10B530001B4A14541878C0B2441CE4B21C70002496
:10B5400014541878C0B2441CE4B21C703478E4B2CD
:10B55000651CEDB2357014541878C0B2441CE4B2C6
:10B560001C70C32414541878C0B2441CE4B21C707C
:10B570006C46247914541878C0B2441CE4B21C7090
:10B580001154054A0B4B11680B401360F7BDC046C0
:10B590002400002075040020680700201602002007
:10B5A000CF050020E806002020020020E906002048
:10B5B00090040020FFFFFFFB8023F7B5334C9B0472
:10B5C000266801901E405FD123685B035CD5304B39
:10B5D0001B181A7A8A4257D08022092719722368C9
:10B5E000D204134323602B4B1D78EDB26A1CD2B2F8
:10B5F0001A70294A57551D78EDB26F1CFFB21F70A3
:10B60000082757551D78EDB26F1CFFB21F705655B5
:10B610001D78EDB26E1CF6B21E70204EB446604628
:10B620003678F6B2771CFFB2077056551D7868461B
:10B63000EDB26E1CF6B21E70BA2656551D78007912
:10B64000EDB26E1CF6B21E7050551878C0B2451C93
:10B65000EDB21D7011541978C9B2481CC0B21870EF
:10B66000022050541978C9B2481CC0B2187080200A
:10B6700050541978C9B2481CC0B2187006235354EC
:10B680002268074B13402360F7BDC04668070020BF
:10B690002400002016020020CF050020E80600202C
:10B6A000FFFFFFFBF7B59C4608AB1D78A023802663
:10B6B0000192DB05DC6876053443DC60DF68224CF0
:10B6C0002D043C40DC60214C032763691A0063466B
:10B6D0003B409F000C239A4317436761A7691C4BAB
:10B6E0003B402B430125A361A3683343A360194B5F
:10B6F0001C6A2C431C62002803D11C6A1648204097
:10B7000003E08024186AE400204318620C2000291A
:10B7100002D1196A814305E0012905D1196A8143E3
:10B7200004200143196208E0022903D1196A814308
:10B730000820F6E7196A08431862FF20596A019A3F
:10B7400081430A435A62F7BDFFFFFFEF000200503A
:10B75000FFFF00FF00000E40FFFBFFFF0D4B0E4AF6
:10B7600099600721186113688B4305390B431360F7
:10B770000A4A936A0B43C7219362094A89005058C9
:10B78000084B0340802000020343535080239B0555
:10B7900013607047C801002030000E4000000E40CA
:10B7A00000E100E0FF00FFFF0E4B0F4AD9600721C8
:10B7B000586113688B4303390B4313600B4A0239FA
:10B7C000D36A0B43C721D362094A89005058094BF9
:10B7D0000340802000020343535080239B051360E5
:10B7E0007047C046C801002030000E4000000E40E7
:10B7F00000E100E0FF00FFFF10B5194C236BDB07F1
:10B800000CD5184A1368002B01D0506898470721BF
:10B81000154A13688B4306390B431360236B9B0750
:10B820000CD5104A1369002B01D090689847072166
:10B830000D4A13688B4305390B431360236B5B0779
:10B840000CD5084A5369002B01D0D06898470721CE
:10B85000054A13688B4303390B43136010BDC04680
:10B8600000000E40C801002030000E400721064AAB
:10B8700013688B4306390B4380211360034A090187
:10B88000136A0B431362704730000E4000000E40F5
:10B8900070B507282AD8164CA24227D80F2B25D8D6
:10B8A00007252840C5003820124C1205A66A864399
:10B8B00030002843A06201200426A56A0140B54358
:10B8C00089002943A162A56A11090B4A2A400A434B
:10B8D000A2620F221340A16A1A02084B0B401343C5
:10B8E000A362A36A1843A062002000E0044870BD70
:10B8F000FF0F000000000E40FFFF00F0FFF0FFFF11
:10B900000181FFFF70B507282AD8164CA24227D81C
:10B910000F2B25D807252840C5003820124C1205CA
:10B92000E66A864330002843E06201200426E56A87
:10B930000140B54389002943E162E56A11090B4AD8
:10B940002A400A43E2620F221340E16A1A02084BBE
:10B950000B401343E362E36A1843E062002000E017
:10B96000044870BDFF0F000000000E40FFFF00F014
:10B97000FFF0FFFF0181FFFF02B471464908490053
:10B98000095C49008E4402BC7047C04603B471464E
:10B99000490840004900095A49008E4403BC7047D9
:10B9A000002243088B4274D303098B425FD3030AFE
:10B9B0008B4244D3030B8B4228D3030C8B420DD311
:10B9C000FF22090212BA030C8B4202D3121209029F
:10B9D00065D0030B8B4219D300E0090AC30B8B42DD
:10B9E00001D3CB03C01A5241830B8B4201D38B038B
:10B9F000C01A5241430B8B4201D34B03C01A524130
:10BA0000030B8B4201D30B03C01A5241C30A8B4272
:10BA100001D3CB02C01A5241830A8B4201D38B025D
:10BA2000C01A5241430A8B4201D34B02C01A524101
:10BA3000030A8B4201D30B02C01A5241CDD2C30973
:10BA40008B4201D3CB01C01A524183098B4201D3EF
:10BA50008B01C01A524143098B4201D34B01C01ADA
:10BA6000524103098B4201D30B01C01A5241C30852
:10BA70008B4201D3CB00C01A524183088B4201D3C1
:10BA80008B00C01A524143088B4201D34B00C01AAD
:10BA90005241411A00D20146524110467047FFE719
:10BAA00001B5002000F0F0F802BDC0460029F7D033
:10BAB00076E7704703460B437FD4002243088B424E
:10BAC00074D303098B425FD3030A8B4244D3030B25
:10BAD0008B4228D3030C8B420DD3FF22090212BAEA
:10BAE000030C8B4202D31212090265D0030B8B4266
:10BAF00019D300E0090AC30B8B4201D3CB03C01A50
:10BB00005241830B8B4201D38B03C01A5241430B2A
:10BB10008B4201D34B03C01A5241030B8B4201D31A
:10BB20000B03C01A5241C30A8B4201D3CB02C01A85
:10BB30005241830A8B4201D38B02C01A5241430AFD
:10BB40008B4201D34B02C01A5241030A8B4201D3EC
:10BB50000B02C01A5241CDD2C3098B4201D3CB0193
:10BB6000C01A524183098B4201D38B01C01A524142
:10BB700043098B4201D34B01C01A524103098B4246
:10BB800001D30B01C01A5241C3088B4201D3CB0031
:10BB9000C01A524183088B4201D38B00C01A524114
:10BBA00043088B4201D34B00C01A5241411A00D2C4
:10BBB00001465241104670475DE0CA0F00D049422D
:10BBC000031000D34042534000229C4603098B429D
:10BBD0002DD3030A8B4212D3FC22890112BA030A25
:10BBE0008B420CD3890192118B4208D389019211A7
:10BBF0008B4204D389013AD0921100E08909C3092C
:10BC00008B4201D3CB01C01A524183098B4201D32D
:10BC10008B01C01A524143098B4201D34B01C01A18
:10BC2000524103098B4201D30B01C01A5241C30890
:10BC30008B4201D3CB00C01A524183088B4201D3FF
:10BC40008B00C01A5241D9D243088B4201D34B001A
:10BC5000C01A5241411A00D20146634652415B105C
:10BC6000104601D34042002B00D54942704763463D
:10BC70005B1000D3404201B5002000F005F802BD82
:10BC80000029F8D016E770477047C0460000000052
:10BC9000200000000000100020001000A50001009E
:10BCA000FF0005000500050005000E013E00FFFF36
:10BCB000FFFFFFFFFFFFFFFFFFFFFFFFFFFFFFFF94
:10BCC000FFFFFFFFFFFFFFFFFFFFFFFFFFFFFFFF84
:10BCD000FFFFFFFF0300880000000000FFFF0500DA
:10BCE0000500050005000F000000FFFF7805400675
:10BCF0001000780540061000780540061000780511
:10BD00004006100078054006100078054006100037
:10BD1000780540061000780540061000FFFFFF0080
:10BD20000F00020014001400FFFFFFFFFFFFFFFFE2
:10BD3000FFFFFFFFFFFFFFFFFFFFFFFFFFFFFFFF13
:10BD4000FFFFFFFFFFFFFFFFFFFFFFFFFFFFFFFF03
:10BD5000FFFFFFFFFFFFFFFFFFFFFFFFFFFFFFFFF3
:10BD6000FFFFFFFFFFFFFFFFFFFFFFFFFFFFFFFFE3
:10BD7000FFFFFFFFFFFFFFFFFFFFFFFFFFFFFFFFD3
:10BD8000FFFFFFFFFFFFFFFFFFFFFFFFFFFFFFFFC3
:10BD9000FFFFFFFFFFFFFFFFFFFFFFFF0204081091
:10BDA000010000000200000002000000040000008A
:10BDB000500251010608520791B1BFA10305540476
:10BDC00012145513181A561992B257A2151758166D
:10BDD000C1C959C5D9E15ADD93B35BA3CDD55CD1B7
:10BDE000090B5D0A0F115E1094B45FA40C0E600D78
:10BDF000363861373C3E623D95B563A5393B643AC0
:10BE0000484A65494E00664F96B667A64B4D684C4A
:10BE1000C2CA69C6DAE26ADE97B76BA7CED66CD221
:10BE20003F416D4045476E4698B86FA84244704305
:10BE3000E5E771E6EBED72EC99B973A9E8EA74E90C
:10BE4000F7F975F8FDFF76FE9ABA77AAFAFC78FB47
:10BE5000C3CB79C7DBE37ADF9BBBC0ABCFD77CD347
:10BE6000EEF07DEFF4F67EF59CBC7FACF1F380F252
:10BE70001B1D811C212382229DBD83AD1E20841F9A
:10BE80002D2F852E333586349EBE87AE30328831D5
:10BE9000C4CC89C8DCE48AE09F538BAFD0D88CD463
:10BEA00024268D252A2C8E2BA07B8FB02729902825
:10BEB000ACAAA9A5A3A69C9A999593968E8D8BB1B1
:10BEC000B2B4B874726C6A696563665C5A5955534A
:10BED000564E4D4B4771E8E4E2D1C9C5D8D4D2CA19
:10BEE000C6CC78171B1D1E2E363A272B2D3539331D
:10BEF0000A0A0A0A0A0A0A0A001BB7000000000020
:10BF00000080510110270000008051010080510184
:10BF100016000000080808080808080808080808AB
:04BF200008080808FD
:00000001FF
